:020000040002F8
:10600000B8510020C1630200C9630200CB630200E3
:10601000CD630200CF630200D163020000000000E4
:10602000000000000000000000000000D363020038
:10603000D563020000000000D7630200D9630200AC
:1060400091670200DB630200F1690200DB6302007A
:10605000DB630200DB63020079650200DB630200A0
:10606000DB630200DB630200DB630200DB63020030
:10607000DB630200DB630200DB630200DB63020020
:10608000DB630200E9670200DB630200DB630200FE
:106090000D680200DB63020011680200DB6302008E
:1060A000DB630200DB630200DB630200DB630200F0
:1060B000DB630200DB630200000000000000000060
:1060C000DB630200DB630200DB630200DB630200D0
:1060D000DB630200DB630200DB630200DB630200C0
:1060E000DB630200DB630200DB63020000000000F0
:1060F00000000000DB63020000000000DB63020020
:10610000000000000000000000000000000000008F
:10611000000000000000000000000000000000007F
:10612000000000000000000000000000000000006F
:10613000000000000000000000000000000000005F
:10614000000000000000000000000000000000004F
:10615000000000000000000000000000000000003F
:10616000000000000000000000000000000000002F
:10617000000000000000000000000000000000001F
:10618000000000000000000000000000000000000F
:1061900000000000000000000000000000000000FF
:1061A00000000000000000000000000000000000EF
:1061B00000000000000000000000000000000000DF
:1061C00000000000000000000000000000000000CF
:1061D00000000000000000000000000000000000BF
:1061E00000000000000000000000000000000000AF
:1061F000000000000000000000000000000000009F
:10620000DFF80CD000F07AF90048004715A302002F
:10621000B851002030B450E8012F93B2C489234410
:106220008489A34228BF1B1B0489A34202BFBFF37A
:106230002F8F002007E0C3EA020340E80134002C5E
:10624000E9D14FF001000A6030BC704750E8012FDF
:10625000C2EA024240E801210029F7D1704730B478
:1062600050E8022F1FFAA2F3C488A34202BFBFF373
:106270002F8F00200DE0C48923448489A34228BFC6
:106280001B1BC2EA034340E80234002CE8D14FF064
:1062900001000A6030BC704750E8022FC2EA224277
:1062A00040E802210029F7D17047034653E8022F46
:1062B000D988B2EB324F4FF0000017BF92B241EADB
:1062C000014142EA014104E05A68B2EB324F08BF93
:1062D000012043E80212002AE8D1704730B4044696
:1062E00054E8000F0D4644E80053002BF8D1156028
:1062F00030BC704730B4044654E8000F40EA010552
:1063000044E80053002BF7D1156030BC704730B41F
:10631000044654E8000F00EA010544E80053002B4E
:10632000F7D1156030BC704730B4044654E8000F14
:1063300080EA010544E80053002BF7D1156030BC1A
:10634000704730B4044654E8000F00EB010544E800
:106350000053002BF7D1156030BC704730B40446B1
:1063600054E8000FA0EB010544E80053002BF7D1DF
:10637000156030BC704770B404464FF0000054E81C
:10638000006F0D68AE4207BF44E80023012044E8D7
:1063900000630E60002B1CBF0020F0E770BC70474C
:1063A00030B4044654E8000F88422CBF451A054615
:1063B00044E80053002BF5D1156030BC7047000055
:1063C0000648804706480047FEE7FEE7FEE7FEE78F
:1063D000FEE7FEE7FEE7FEE7FEE7FEE715680200E0
:1063E000016202002DE9F05F0546002092469B46BF
:1063F00088460646814640241BE0284641464746DB
:10640000224600F06BF853465A46C01A914110D309
:1064100011461846224600F016F82D1A67EB0108BF
:106420004F4622460120002100F00DF817EB00092D
:106430004E41201EA4F10104DFDC484631462A46C5
:106440004346BDE8F09F202A04DB203A00FA02F11F
:10645000002070479140C2F1200320FA03F3194352
:10646000904070470048704798FE020040EA0103E0
:106470009B0703D009E008C9121F08C0042AFAD2FA
:1064800003E011F8013B00F8013B521EF9D27047BE
:10649000D2B201E000F8012B491EFBD27047002266
:1064A000F6E710B513460A4604461946FFF7F0FF13
:1064B000204610BD421C10F8011B0029FBD1801A98
:1064C000704730B504460020034600E05B1C934251
:1064D00003D2E05CCD5C401BF8D030BD202A04DB49
:1064E000203A21FA02F00021704721FA02F3D0404D
:1064F000C2F120029140084319467047064C074DEF
:1065000006E0E06840F0010394E807009847103483
:10651000AC42F6D3FFF778FEEC0603000C0703004D
:1065200070B58C1810F8015B15F0070301D110F855
:10653000013B2A1106D110F8012B03E010F8016B82
:1065400001F8016B5B1EF9D12B0705D40023521E05
:106550000DD401F8013BFAE710F8013BCB1A921C6D
:1065600003E013F8015B01F8015B521EF9D5A1426B
:10657000D8D3002070BD00002DE9F04F00268DB06B
:10658000DFF8A081B14604964FF4807501243746A8
:106590000596284605F014F938B1D8F804032042CE
:1065A00003D0284605F002F926432D1D64007F1C08
:1065B000ADB2082FEDD34FF4BE74204605F000F9BC
:1065C00048B1204605F0F2F846F0004604AA022140
:1065D000002005F0D5F8544C16F0FF0F15D0012718
:1065E000002537420DD008EB8501D1F81005D1F810
:1065F0001015C0F3052054F82520C1F3014102B164
:1066000090477F006D1C082DEBD3002E7EDA002012
:10661000CDF82890411E0DF1100B07AACDF82C9053
:1066200042F82010401C91460228F9D300252E463E
:10663000A11911F8607F91F9000027F0C008401CF3
:1066400040D007A9404604F0B4F940B34FEA971A86
:10665000404602F043F854F820701FB1BAF1030F1E
:1066600003D006E0BAF1030F2CD10AA9404604F08A
:10667000A8F902A8CDF8088005F026F8029900EBE9
:106680008100D0F8000704A9C0F301400290404601
:1066900004F08FF90028029802D0022802D011E0FD
:1066A00003280FD1BAF1030F08D10298022833D082
:1066B0000221404604F0E2FF6D1CEDB217B15146D5
:1066C0004046B847761C042EB2D3002D21D001AA33
:1066D0000221002005F054F800205A460DF1040173
:1066E00052F8206051F82030B34217D000200AAE93
:1066F0004FEA090351F8207042F8207056F82070D4
:1067000043F82070401C0228F4D300E001E0002D83
:106710008CD10DB0BDE8F08F0321CAE7401C0228E0
:10672000DED3F6E700600040F428002000F01F02EE
:10673000012191404009800000F1E020C0F8801262
:10674000704700F01F02012191404009800000F1D4
:10675000E020C0F80011704700F01F0201219140B5
:106760004009800000F1E020C0F80012704749079E
:10677000090E002806DA00F00F0000F1E02080F892
:10678000141D704700F1E02080F8001470470000ED
:1067900070B54FF48076304604F04AFA114CB505D6
:1067A00060B1304604F04BFA0120C5F80803607967
:1067B00020B9012060712168002088474FF482765B
:1067C000304604F035FA00280AD0304604F037FA93
:1067D0000220C5F808032168BDE870400120084781
:1067E00070BD0000B822002007480021C0F8401109
:1067F000C0F84411C0F84811C0F84C11C0F800119D
:10680000C0F8041108F09ABB0010014008F0E4BA87
:1068100005F080BD30B54FF0805000228300D0F8E5
:106820003011C3F80C21C3F81021624B1A60624B7F
:106830001B68624C2360604B1B1D1B68241D23607A
:106840005D4B08331B68241D23605B4B0C331B68B6
:10685000241D2360584B10331B68241D2360564BA6
:1068600014331B68241D2360534B18331B68534C8F
:1068700020342360504B1C331B68241D23604E4B77
:1068800020331B68241D23604B4B24331B68241DBD
:106890002360494B28331B68241D2360464B2C334F
:1068A0001B68241D2360444B30331B68434C403429
:1068B0002360414B34331B68241D23603E4B383327
:1068C0001B68241D23603C4B3C331B68241D236044
:1068D000394B40331B68241D23600124082902D151
:1068E000D0F8343113B1082904D006E0354B3449CF
:1068F000196005E0D0F8343113B1082904D006E05E
:10690000314BFB21196005E0D0F8343113B108296F
:1069100008D00EE090F858322C48016863F3030168
:10692000016002E0D0F834311BB929494FF40070FE
:10693000086028480168C90702D06FF001010160B2
:106940002548016841F470010160BFF34F8FBFF328
:106950006F8F4FF01021D1F80002002803DBD1F82F
:106960000402002822DA1D4B1C601D480468002C1C
:10697000FCD01224C1F800420568002DFCD0C1F8FB
:10698000044201680029FCD01A6001680029FCD08B
:10699000BFF34F8F10487C380168124A01F4E06160
:1069A00011430160BFF34F8F00BFFDE70F490E4851
:1069B000086030BD380500400404001020C50040C8
:1069C000488103008C56004018F50040E40E00405A
:1069D000409602400004004088ED00E004E50140DC
:1069E00000E401400400FA050090D003DC230020FD
:1069F0000148006800470000C022002002E008C8EB
:106A0000121F08C1002AFAD170477047002001E028
:106A100001C1121F002AFBD170470000012120286C
:106A200003DA81400548014003E0402802DA2038BB
:106A3000814009B10120704700207047FC06FFBD6E
:106A400010B560B159B102780B785208B2EB530F10
:106A500005D10622401C491CFFF733FD08B1002078
:106A600010BD012010BD800701D00020704701201B
:106A70007047C3688B4206D811440069491E8142A1
:106A800001D8012070470020704710B50122022173
:106A9000002001F027FC08B1072810D107220221AD
:106AA000012001F01FFC08B1072808D100210A22AB
:106AB000084601F017FC08B1072800D1002010BDDE
:106AC00010B550B10A480321008801EB004009A12C
:106AD00005F066F807F0B2F803E00321094800F07A
:106AE000A0FC002803D0BDE8104000F0CBB810BDDA
:106AF00024240020457261736520626F6E647321E7
:106B0000000000005424002070B58CB015460E46DD
:106B100000236C46C3F10F01415CE1545B1C102B58
:106B2000F8D30D2104F11000FFF7B9FC0020C0F1EB
:106B30000F02315C2244401C11740328F7D36846CD
:106B400046DF0020C0F10F01214491F820102954A4
:106B5000401C0328F6D30CB070BD022001F0C4BA6B
:106B60000149097900F0F0BD8022002070B50024B1
:106B7000064D06E06868012110F8340005F0B4FC09
:106B8000641C28788442F5D3002070BDC822002000
:106B9000F8B515460C460646052A01D20720F8BD71
:106BA00005F09AFD18B905F05DFD0028F7D11249EE
:106BB00000224E600C708D60C1E90422C1E90622FA
:106BC0000E4D0DE006EBC4002968009181788DF828
:106BD000011000780A4A694605F0D2FC0028DED18F
:106BE000641EE4B2EED2BDE8F84004480021054A34
:106BF000001D00F099B80000C822002014FB02001C
:106C0000AD960200298B020072B605F07FF800BF36
:106C100004F0B6FE0028FBD1104C0121208801EBC6
:106C200000400FA104F0BCFF10480068C00700D06E
:106C300000BE2088022101EB00400DA104F0B0FF4E
:106C4000BFF34F8F0948E43801680D4A01F4E06151
:106C500011430160BFF34F8F00BFFDE724240020E4
:106C6000466174616C206572726F7200F0ED00E035
:106C700053797374656D207265736574000000004C
:106C80000400FA050EB500210091CDE901106A4615
:106C900044F20100FFF7B8FF0EBD000070B50228F6
:106CA0000DD1084C032508A1208805EB004004F015
:106CB00077FF208810A105EB004004F071FF012050
:106CC00070BD000024240020506F776572206D6134
:106CD0006E6167656D656E742077616E7473207484
:106CE0006F20726573657420746F20444655206D63
:106CF0006F64652E00000000506F776572206D6133
:106D00006E6167656D656E7420616C6C6F7765642C
:106D100020746F20726573657420746F204446552B
:106D2000206D6F64652E0000074B9B7823B12AB15C
:106D300020B10068037C1BB1082070470720704712
:106D40004174426100207047D029002070B507F0DF
:106D500067FA104800240B21047044700E4D8170B6
:106D600014206C602C706C70FFF7E0FC072114207D
:106D7000FFF7FDFC1420FFF7E4FC0848046007213E
:106D80001120FFF7F4FC0548001F0068A8600020F0
:106D900070BD0000D0290020E82200200815014025
:106DA0002DE9FC47DFF8789099F8023073B368B3A7
:106DB000052902D20720BDE8FC87436933B3437C31
:106DC000012B25D0002704460025884616468DF85D
:106DD0000050684600F038F801A808F045FBC8B13B
:106DE000012101700F4944600968C0E90218C0E937
:106DF00004769DF8040089F801009DF8000000F079
:106E000047F81420FFF7A8FC2846D4E70820D2E76B
:106E10000F46D8E704259DF8000000F039F8F3E7A5
:106E2000D0290020041501400649897839B130B1D4
:106E3000416921B100210174022108F05BB80820EA
:106E400070470000D029002030B5EFF3108172B6F2
:106E50000D4A9468012324B10370002900D162B661
:106E600030BD93604FF0E023D3F88051074C2540AC
:106E70001560C3F88041D3F8844154605A17C3F8B1
:106E8000842100220270E8E7DC2A0020FC06FFBD16
:106E90000B498A68002A11D000280FD1EFF3108027
:106EA00072B60B684FF0E022C2F800314B68C2F8AE
:106EB000043100228A60002800D162B670470000C9
:106EC000DC2A002070B5054608680C46411C04D039
:106ED00004F02FFC206804F0BDFB6068411C02D068
:106EE000002104F0A5FB2968A069C1F82405607D94
:106EF000227D29681043C1F86C05D4E90012286886
:106F0000C0F81425C0F80C15207D012814D1A06804
:106F1000411C02D0002104F08BFBE068411C04D02E
:106F200004F007FCE06804F095FBD4E9021228683D
:106F3000C0F80825C0F8101570BD70B50546086882
:106F40000C46411C04D004F0FEFB206804F08CFBCE
:106F50006068411C02D0002104F073FB2968A0691D
:106F6000C1F82405607D217D2A680843C2F86C05BC
:106F7000D4E900122868C0F80C15C0F81425207D4B
:106F8000012814D1A068411C02D0002104F059FB53
:106F9000E068411C04D004F0D6FBE06804F064FB18
:106FA000D4E902122868C0F80825C0F8101570BD91
:106FB00003F00CB92DE9F047074600888EB08046F3
:106FC00002F0FAFD824604462D4800252A46017843
:106FD000404600F0D1FB7879400734D501254FF6C3
:106FE000FF7603AB2A460721504606F089F80100D8
:106FF00004D0404607F00CFB00252BE0B14631469B
:10700000049802F02DFD064648450FD0044601467F
:10701000404602F0BBFD4046FFF7A2FD30B94046B6
:1070200007F0C8FA4046FFF79BFD48B1224607210A
:10703000504606F0DBF8010003D0404607F0E8FABE
:1070400000254E4506D0404606F03EFA10B15046A7
:1070500002F09EFD02208DF81800ADF81A807879B4
:10706000400701D5012000E002208DF820008DF8B6
:10707000215006A801F0CCFE0EB0BDE8F08700005C
:10708000802200202DE9FC47002517880646158040
:1070900090F82D001446894630B13A4621464846BC
:1070A00000F094FB051E09D1B0784FF00C0A18B31C
:1070B0002088C846001DB84202D95046BDE8FC876A
:1070C000684679DF0028F9D12088032108F80010EC
:1070D00020881921401C80B2208008F800102088E8
:1070E000401C80B2208000EB0801BDF8000008F0D1
:1070F000E9F8218808442080F0780222C8B121886C
:1071000096F9033001F1030C4846BC45D5D84254EA
:1071100021884FF0010C491C89B2218000F801C080
:107120002188491C89B2218009F801302088401C3F
:1071300020807068B8B1218890F9003001F1030C0B
:107140004846BC45B9D8425421880A22491C89B214
:10715000218042542188491C89B2218009F80130DC
:107160002088401C2080308950B1CDE900474B4633
:107170000622022106F1080008F08EF9051E9DD1B5
:10718000308A50B1CDE900474B460722032106F172
:10719000100008F081F9051E90D1308B50B1CDE977
:1071A00000474B461522142106F1180008F074F927
:1071B000051E83D1306A30B13B462246494601F074
:1071C00048FB051EDBD1706A30B13B46224649467A
:1071D00003F0AAF9051ED2D196F82C0038B13B462F
:1071E00022464946304607F0B9FA051EC7D1307825
:1071F00038B13B4622464946304603F01BFA051E8D
:10720000BDD128465AE718B504460020ADF8000065
:1072100013466A46204600F006F8002802D0BDF862
:107220000000204418BD70B588B182B100241588D3
:1072300003E0065D641C3444A4B2A54203D80619D9
:1072400076789E4201D08C42F3D38C4201D3002049
:1072500070BDA11C1180005D401E80B270BD80F821
:10726000301070472DE9F0410E00044606D02CB1D5
:1072700096F87A000025012803D006E00E20BDE82C
:10728000F08196F89800012821D04FF00108A570F0
:107290002C2206F17801201DFFF7E8F884F8305021
:1072A000D6F8A4006063D6F8A800A0634FF6FF707C
:1072B000A4F8A80004F19400C4F8A400C4F8AA50EB
:1072C000A4F8AE5084F8B050207810B104E0072044
:1072D000D5E7FF2084F8540004F155011F27C4F8B6
:1072E0009410A4F8987004F198023046FFF7CAFE93
:1072F0000028C4D116F13C0F0ED004F17401C4F87B
:107300009C10A4F8A07004F1A00206F13C00FFF765
:10731000B9FE0028B3D103E0C4F89C50A4F8A050F3
:1073200084F85180208BA4F8480084F83C802564C0
:1073300084F8505060696064464604F13C020021C4
:1073400004F1540072DF002899D1267097E710B538
:107350000288102A1BD0112A20D0262A1DD1007A9B
:107360000C46012801D0022817D1A0780521401C25
:10737000B0FBF1F201FB1201204600F052F80028A8
:107380000BD0A16B002908D0BDE810400847C27B94
:10739000012A02D18088A1F8A80010BD0C46002166
:1073A00084F8B2108088B4F8A8108842F5D120790A
:1073B0000028F2D10121DFE710B50C46022801D0E8
:1073C000032810D1607800280DD000206070A178CB
:1073D000204600F026F8002805D0A16B002902D035
:1073E000BDE81040084710BD10B5044690F85400A1
:1073F00074DF012084F8B200002084F8B40084F81F
:1074000050000621204601F009FF002808D1A1788C
:10741000204600F006F810B1A16B01B188470020AA
:1074200010BD2DE9F05F044600780F4638B1A77013
:10743000002003F007FF012620B1667007E1082055
:10744000BDE8F09F0025C4F8AA50A4F8AE5084F817
:10745000B050A07910B1A078012806D0E07968B1C9
:10746000A078012801D0022808D1616B21B184F8ED
:10747000B1600820884701E084F8B15004F1AB0105
:1074800000200A5C0AB1304603E0401C0628F8D30D
:1074900000204FF002084FF0030B012F06D0022FFF
:1074A0000CD0032F0FD0042F15D110E0A17929B1F2
:1074B00094F8241011B908B130460DE0E17911B10A
:1074C00008B1404608E0207A08B1584604E0607AE6
:1074D00008B1042000E02846A070616B41B1032888
:1074E00001D0042804D1607910B194F8B200A0B1A1
:1074F00084F8B35004F13C0018210746FEF7CFFF93
:1075000004F12C0084F83C60814606F009F958B17A
:1075100094F82C0084F8510008E084F8B45084F802
:10752000B36007208847E5E784F8516094F82400A9
:1075300050B1484606F0F4F820B194F8280084F8D9
:10754000520001E084F8526084F85050A27804F1AF
:10755000AA0104F194094FF0060A052A60D2DFE877
:1075600002F078030F223F0084F83160C4F8A45081
:10757000C4E9101584F83C808020A4F8480051E04C
:1075800084F8318094F82420384612B10722027022
:1075900001E080F800B0228A8281C4F8A4504160E2
:1075A000E168B9603EE06069B860208BB88194F80A
:1075B00024003D4610B184F83CA001E084F83C6012
:1075C000204607F02DFF40B185F8148004212046A5
:1075D00001F024FE20BB05211EE084F831B01DE03F
:1075E000E069B860208CB88194F824003D4610B161
:1075F00084F83CA001E084F83C60204607F010FFCE
:1076000048B185F814800421204601F007FE38B9FE
:1076100084F831A002E0042184F83110C4F8A49069
:10762000A07878B13A4604F15400D4F8A41072DF7F
:1076300000287FF405AF94F8301094F8540073DFFD
:107640000028F6D1616B11B194F831008847002011
:10765000F6E684F83150F5E770B5040012D0014623
:107660001C221448FEF702FF1248134D05602068E3
:1076700050B17ADF002806D120680168296040688F
:10768000686005E00E2070BD0B487BDF0028FAD152
:1076900008484FF6FF711438084A20F8041B0549C2
:1076A000343901600021FFF73FFB0028EBD00320B5
:1076B00070BD0000AC25002040220020B9F302007C
:1076C00010B5044600F078F8002805D02146BDE842
:1076D0001040024803F0D1B810BD0000D8250020AA
:1076E00070B515460E46044607F0A6FE002809D0E0
:1076F000054800EB840080692A463146BDE87040A9
:1077000001F0CABD70BD0000C825002070B5054657
:10771000002400F051F838B12946044803F0ADF8D0
:1077200008B1022400E00124204670BDD4250020C9
:1077300010B51821034803F07BF8182800D0C0B218
:1077400010BD0000C825002070B505460C4608464F
:1077500007F072FE60B1284600F02EF840B10548EF
:10776000294600EB8400BDE87040183003F085B86E
:10777000002070BDC825002070B5054614460E4691
:10778000084607F059FE002812D0284600F014F8E9
:1077900000280DD00748294600EB860018301CB1A0
:1077A000BDE8704003F074B8BDE8704003F025B840
:1077B00070BD0000C8250020142801D300207047A8
:1077C0000146014803F059B8CC2500207CB5054698
:1077D00008880C460930904201D90C207CBD6846CF
:1077E0006DDF0028FAD121880820685420881B21E9
:1077F000401C80B2208029542088401C80B2208008
:107800002844DDF801100160BDF805108180208852
:10781000801D80B220809DF80010490800D0012111
:1078200029542088401C208000207CBD10B503F026
:107830000FFA002809D105484FF0030C00DF00289B
:1078400003D1BDE8104003F067BA10BDB82800208E
:1078500018B103490860002070470E2070470000EF
:10786000A022002010B54FF0FF3100203DDF00289E
:107870000BD1B1213CDF002807D104484169012028
:107880008847022004F066FB002010BD9C280020E1
:10789000044810B50068416900208847BDE81040E1
:1078A000FFF7E0BFA022002030B58FB005461C21B5
:1078B00001A8FEF7F4FD0024142109A80894FEF79E
:1078C000EEFD9DF82000009420F00F00401C20F0F9
:1078D000F00010308DF820009DF82100029420F077
:1078E0000F00401C20F0F00010308DF821009DF8B2
:1078F0002200049420F00600801C8DF822009DF8E0
:10790000040009AA40F028008DF8040008A8CDE979
:107910000540079428788DF83A000320ADF8380028
:107920009DF80000ADF82C4020F00F00401C20F026
:10793000F00010308DF800009DF80100ADF82E40E9
:1079400020F00F00401C20F0F00010308DF80100F6
:107950009DF802000D9420F00600801C20F0080025
:1079600040F011008DF802000EA809901720CDF804
:1079700028D0ADF830006888AB1D01A9AADF0FB090
:1079800030BD000010B5164C86B01ECC8DE81E0030
:1079900020B3144C4FF6FF71A18000686061002095
:1079A000607620762046FFF753FF002814D101208F
:1079B0008DF812004FF65960ADF81000A21C04A912
:1079C0000120A8DF002807D12146684662DF002891
:1079D00002D12046FFF768FF06B010BD0E20FBE77E
:1079E000F4FA02009C28002010B500280FD001886E
:1079F000204C502926D00BDC10291DD0112906D18E
:107A0000A1888088814202D14FF6FF70A08010BD0E
:107A1000512913D05329FAD1C088E1888842F6D180
:107A2000607E0028F3D0FFF733FF0028EFD06169B4
:107A3000BDE81040022008478088E7E7BDE8104015
:107A400005F05EB930F8061F62899142DFD14189A5
:107A50000229DCD10C3000F0FBFA07492076032222
:107A60000988BDE8104002EB0143024603A1184615
:107A700004F09AB89C2800202424002052656365F5
:107A80006976656420696E6469636174696F6E20EC
:107A90007374617465202564000000002DE9F041D5
:107AA0000546007B042601272D4C012811D0022811
:107AB0002CD00226287B314600F08AF818B12068C5
:107AC000416903208847206841690220BDE8F041F0
:107AD000084720684FF00008817E49B10621012047
:107AE00000F076F8002839D0206841690320EDE7DE
:107AF00047760121084600F06BF800282ED0226856
:107B0000112882F81980D5D10626D3E76A7B142A7A
:107B100020D8FAB1DFF84C8005F10E0108F104001D
:107B2000FEF7A4FC697BC8F8181021684046897EDE
:107B30000029BFD1A0F10C010A68011F904758B17C
:107B40000F28B7D108480949008807EB004004F026
:107B500027F8AFE70526ADE720688776BDE8F08116
:107B6000A0220020C42800202424002040FF02007E
:107B700070B5154900250A68002A24D04A68002AF1
:107B800021D00831904708281DD0104C00282068CB
:107B900085760ED00621022000F01AF818B1206870
:107BA000416903208847206841690220BDE8704090
:107BB00008470121022000F00BF8002803D02068BC
:107BC00041690320F2E770BDB8280020A022002000
:107BD00086B00323ADF8003020238DF814308DF8E3
:107BE000150000220E48019202928DF81610C188ED
:107BF000ADF8041002218DF8061005A90491ADF826
:107C00000820CDF80CD0808801A9AEDF002804D16F
:107C1000BDF80010032900D00C2006B0704700000A
:107C20009C2800200F4A0321128801EB024268B110
:107C300001280ED00B4A01210228128801EB0242D2
:107C40000AD0032810460AD007A109E0104610A167
:107C500006E010461AA103E0104622A100E030A180
:107C600003F09EBF24240020556E6B6E6F776E204C
:107C70006576656E742066726F6D20626C655F64F8
:107C800066755F627574746F6E6C6573732E000039
:107C900044657669636520697320707265706172EE
:107CA000696E6720746F20656E74657220626F6FF5
:107CB000746C6F61646572206D6F64652E000000E6
:107CC0004465766963652077696C6C20656E7465C0
:107CD0007220626F6F746C6F61646572206D6F6487
:107CE000652E00005265717565737420746F206590
:107CF0006E74657220626F6F746C6F616465722060
:107D00006D6F6465206661696C6564206173796E6E
:107D10006368726F6E656F75736C792E000000007A
:107D20005265717565737420746F2073656E64207D
:107D30006120726573706F6E736520746F20636C61
:107D400069656E74206661696C65642E00000000D0
:107D500038B50446008821281CD013DC102822D115
:107D6000072000F0E1FA08B1FEF78CFF1048A18867
:107D70000180104802F0E4FE002814D0BDE838402D
:107D8000FEF780BF3B280FD056280CD1A0881321C6
:107D900076DFF1E700200090A08869468FDF002899
:107DA00001D0FEF76FFF38BDA088132176DFE3E72F
:107DB000202200204824002010B51A4C0188606859
:107DC00010290ED011292BD1401E606028D1FEF75A
:107DD0005CFE002824D02168002921D0BDE8104095
:107DE0000847D0B900210122084600F07BFA08B10B
:107DF00007280FD107220221012000F073FA08B1F1
:107E0000072807D104220221002000F06BFA20B1DC
:107E1000072802D0216801B188476068401C606073
:107E200010BD0000382200202DE9F04701883B4EAC
:107E300040F2F3194FF6FF7510291BD011293ED0DF
:107E4000122954D0502946D1C188F289841D91420B
:107E500041D1618902293ED18688304601F058FF20
:107E6000050038D004F10C0000F0F6F8A8B329465C
:107E700030464EE0C17B8788044601292BD1A846B5
:107E8000284601F045FF050017D02F8000202872FA
:107E9000234843464A460168C5F80A104068C5F8B9
:107EA0000E0004F1100105F10A0001F0FDFF6872F7
:107EB000F08900280FD129462AE0042013E08088A9
:107EC00001F026FF040006D06068FEF7ADFF08B1A0
:107ED00006F082FB2580BDE8F087FFE76868FEF7C3
:107EE000A3FF0028F7D0BDE8F04706F075BB8788F0
:107EF0000646384601F00CFF0400ECD02B464A46FB
:107F000006F1080104F10A0001F0CEFF607221467B
:107F10003846BDE8F04700F0E3BC0000AC25002087
:107F2000402200202DE9F04F0746858802883D4811
:107F3000012197B08346102A09D0112A49D01A2A64
:107F40006CD1387AB1EB101F45D2012244E0354C98
:107F5000083CA068C0430B9061680BA802F0B1FC1C
:107F60000B990CA800F056FC2C220CA96846FEF7D1
:107F70007DFA0026E946A04610E000BF09EB460066
:107F80005FF00004B0F804A008EB84005146001D27
:107F900002F033FC641C1D2CF6D3761C0098B04212
:107FA000ECD8142D05D317B00420BDE8F04FFEF730
:107FB00069BE2946584602F06BFC294608F10400C8
:107FC00002F066FCF87B012828D016482946001DDF
:107FD00015E029461AE000220221B1EB101F01D260
:107FE000012600E000260F49083901F11000041DA8
:107FF000294682B102F04CFC36B12946204617B022
:10800000BDE8F04F02F044BC2946204617B0BDE859
:10801000F04F02F0F2BB02F0F0FBF5E717B0BDE85D
:10802000F08F0000D025002010B5044607480078E6
:1080300000280AD0204601F099FC204606F026FCD4
:108040002046BDE8104001F033BA10BD7022002078
:108050000078C0F340007047007800F001007047DE
:108060000149085C70470000ACF90200084908B5F6
:10807000085C0090684603F019FBD0F810050099E1
:10808000C84010F0010000D0012080F0010008BDC0
:10809000ACF902002DE9FC410646C0074FF000058F
:1080A0000ED0104F00240122385D009500231146A8
:1080B000019503F047FA641C042CF4D300F04EF849
:1080C000B0070DD5074E0024361D0022305D032376
:1080D00000951146019503F035FA641C042CF4D385
:1080E000BDE8FC81A8F90200094908B5085C0090C8
:1080F000684603F0DBFAD0F80425009B0121994083
:1081000021EA0203C0F808351140C0F80C1508BD7B
:10811000A8F902000249085C012103F01EBB00001F
:10812000A8F902000249085C002103F016BB000018
:10813000A8F90200084908B5085C0090684603F0F9
:10814000B5FAD0F804050099C84010F0010000D03D
:10815000012080F0010008BDA8F9020010B500243C
:108160002046FFF7D7FF641C042CF9D310BD10B5CF
:1081700000242046FFF7D6FF641C042CF9D310BD61
:1081800010B50246064B4FF0FF3000215C5C944274
:1081900001D1084610BD491C0429F7D310BD0000C9
:1081A000ACF9020070B50C4E0C004FF000053060C9
:1081B0000BD0012000F06AF808B1022004E0002092
:1081C00000F064F800B10B202070706810B9FEF761
:1081D0005CFC0546284670BD3822002010B5002002
:1081E00000F0D4F908B1062806D1012000F0CEF93C
:1081F00008B1062800D1002010BD00002DE9F0478D
:108200000D468146FFF7BCFF0446042836D2DFF84E
:1082100074801B481C4EA8F10C0725B3012D0ED00D
:10822000022D2BD104EB440030444578002D25D09D
:10823000B968002922D02846BDE8F047084704EB7A
:108240004401755C0E44717849B10E4A4FF4004107
:10825000093A8068FEF7A4FD08B987F80390B17861
:1082600008F80410E2E78068FEF7DEFD04EB440145
:10827000314418F804008D78A842D7D0BDE8F087C3
:10828000B0F90200342200204C250020042801D23D
:10829000FFF7ECBE002070470146104810B500887B
:1082A000042907D007290ED00A2915D1BDE81040AE
:1082B00006F0D6BA132176DF0CE000280CD0BDE81A
:1082C0001040FEF7DFBCA0F57F41FF3904D1044820
:1082D000FFF78AF80828F0D110BD00002022002006
:1082E0005424002070B50023042810D20D4D00EB5B
:1082F0004004012A02D101290CD00022094E00EBD2
:108300004000304461B1012906D0022906D007237C
:10831000184670BD0E30C2B22A55F9E74270F7E731
:108320008270F5E74C250020044A014600201279AE
:10833000D20702D0084600F04DB87047282200202E
:1083400070B506461E480024C0E90161B00720D57B
:108350000025012211462846FFF7C4FF6D1C044684
:10836000042D02D2002CF4D013E094B940F26662DE
:1083700004211448FEF70CFC04000AD1FEF7F6FBBA
:10838000040006D10F48104A0021001FFEF7CCFC64
:108390000446F00712D00120FFF77CFE74B90948AB
:1083A0000A4A00210C38FEF7BFFC040006D105483C
:1083B000074A01210838FEF7B7FC0446204670BD85
:1083C00028220020BCF90200598602003D9F0200CD
:1083D0005B6B02002DE9F05F6A4C05460026607871
:1083E000B34618B184F801B001F090FD664F4FF428
:1083F0007A694FF4C87A4FF00108182D62D2DFE88D
:1084000005F0AC0C0C31404D62676B746B74BE7D33
:108410007D7D7D7DACAFB2B5BEBE0020FFF78AFE8C
:1084200000284FF0000008D0FFF774FE022D02D1A3
:108430004FF4E16008E0484606E0FFF773FE022DC6
:1084400001D1C82000E05046410CC0034FF4FA723D
:10845000801841F10001257052000023FDF7C2FF92
:1084600001462AE00020FFF765FE00284FF00000DB
:1084700004D0FFF74FFE4FF44870E5E7FFF752FED8
:10848000DFE70020FFF756FE00284FF0000002D083
:10849000FFF740FECFE7FFF745FED4E70020FFF7E8
:1084A00049FE00284FF0000002D0FFF733FE01E044
:1084B000FFF738FE257041F69A1100223868FEF762
:1084C0006FFC064646E00020FFF70EFE257008E030
:1084D000002051E025703DE084F801800120FFF785
:1084E00003FE002240F6CD41E8E784F80180012038
:1084F000FFF7FAFD00224FF48041DFE77868FEF7CE
:1085000093FC0646D5F1110000D02EB10220FFF7F2
:1085100001FE84F802B01DE0012816D980B2C821FE
:108520004843C117C90341EA5041C0034FF4FA72EE
:10853000801841F1000152000023FDF753FF01466E
:1085400000227868FEF72CFC06460220FFF7EAFDC1
:1085500084F802803046BDE8F09F01F0D7FCB9E70F
:1085600001F0D4FCB4E701F0D1FC04E001F0CEFC52
:108570000020FFF7D7FD0120FFF7D4FDAAE7FFF7A2
:10858000F6FDA7E728220020B0F90200012106F03D
:10859000EBBF00002DE9F8430546861C00208DF84E
:1085A000000090460F464FF001096846FEF74CFC6C
:1085B0001B4C20683860D4E90001401AA16804F21D
:1085C0001C47081A0EE00121384602F074F901F048
:1085D00053FE0146384602F06EF9D4E90001401A14
:1085E000A168081A401C8642EDD8B8F1000F03D0EC
:1085F000052065F3891002E0062065F39F50A2680C
:108600002168114004EB8101C8602068304420607B
:108610009DF80000FEF73CFC4846BDE8F8830000EA
:10862000942D002030B482680468531C8360A154E8
:10863000D0E901128A4202D330BC02F030BC30BC17
:1086400070470000034803C8814201D101207047F0
:1086500000207047942D002000780221FFF7CEBD46
:10866000032805D10349A9200860002003F072BC4B
:10867000704700002005004005494FF0FF320828F0
:1086800041F8202002D3084480F8582070470000A9
:10869000F4280020F0B54FF0FF3512B10023082672
:1086A00001E008230C260C4C05E000BF54F82370B1
:1086B0007F1C04D05B1CB342F8D32846F0BD2618BB
:1086C0005DB286F8305044F82310002AF5D1E11845
:1086D00081F85800F1E70000F4280020024908441E
:1086E00090F9300070470000F428002070B504466F
:1086F0004FF6FF750A462846AC4208D14FF4807405
:108700002146104605F064F9A04209D070BDFF2C47
:10871000FCD82146104605F04EF908B1204670BD40
:10872000284670BD70B5084C050009D0103421688A
:10873000002907D008682060496828468847F6E77E
:108740000834F4E770BD0000E0280020054A01214C
:1087500020B1012805D19170FFF7E4BF51700020CE
:10876000FAE77047E02800202DE9F05F26484168CD
:10877000F1B3DFF898B00E688146DBF800408768F7
:108780008078E11B21F07F45ED1CB0B9DFF88080D7
:108790004FF48030C8F84403C8F804031120FDF7F3
:1087A000C5FF1120FDF7CDFF4FF0010AC8F800A06A
:1087B0002F2003F091FE89F802A0B54200D2354681
:1087C000124BE8193C3320F07F401860DBF80010B2
:1087D0005A46091B21F07F41001B20F07F40C91C35
:1087E00081420FD9106818602F2003F075FE00E059
:1087F00004E0BDE8F05F1120FDF7AEBFBDE8F05F1B
:1088000005F00EBDBDE8F09FE822002004150140F0
:108810000010014073B58CB00646002000900D9802
:1088200080B100246D4621460DA802F026F830B133
:10883000009805EB400084800098401C0090641C68
:10884000142CF0D32C2269463046FDF70FFE0EB0F3
:1088500070BD2DE9F04117880646B81D14460D4637
:10886000984202D90C20BDE8F08131880722062900
:108870000AD34FF4486C4FF6FF73614501D9994212
:1088800002D17088062801D21046ECE7604501D974
:108890009842F9D1994203D0984201D08142F3D84D
:1088A0000520E85520881221401C80B220802954E0
:1088B0002088401C80B220804119308806F002FDDB
:1088C0002188084480B220804119708806F0FAFCA3
:1088D0002188084420800020C5E7FEF7D3B90000B6
:1088E00038B54A7A0F4B62B100220A7259690029E1
:1088F00006D001228DF80020ADF8020068468847B6
:1089000038BD0A7A62B19B684C6802461946204617
:10891000FEF746FA0028F3D0BDE8384005F05CBE0B
:108920005B68F1E7AC250020F0B585B016460F4630
:1089300004461D4614220B496846FDF797FD0A4878
:108940008DF80870ADF80240ADF80A608DF80C5053
:10895000017800222046FEF70FFF684600F058FA23
:1089600005B0F0BDC8FA020080220020F0B587B043
:10897000074600200490ADF810100590ADF81210D5
:108980000190029001AA04A9384690DF060022D087
:1089900003F048FD114C0346012520883A4605EBBB
:1089A00000400F4903F007F9BDF8042012B9BDF8E3
:1089B000060038B12088BDF8063005EB004009A15B
:1089C00003F0F9F8BDF808202AB12088154905EB15
:1089D000004003F0E9F807B03046F0BDF423002072
:1089E0009CFE02005468652072657175657374653C
:1089F000642054582F5258207061636B6574206C4A
:108A0000656E67746820697320746F6F206C6F6E79
:108A1000672062792025752F2575206F6374657432
:108A2000732E0000E8FE020030B5044685B0002138
:108A30001B4804F0C0FF00282FD00025204600F07E
:108A4000C4FE68B1112812D086281BD0A0F5405171
:108A5000023903D00146204605F0C6FD294607E04D
:108A600005B029462046BDE8304001F0E3BB0121B6
:108A7000204601F0DFFB05B00021BDE8304008488A
:108A800004F0CDBF142207496846FDF7EFFCADF8AE
:108A90000240684600F098F9E0E705B030BD0000FC
:108AA00049220020F0F902007FB50C4610B10120E8
:108AB00004B070BD2079002638B141F61D5501285B
:108AC0001BD0022826D00F20F2E702202071029648
:108AD0000396E0680190694601A805F0FDFA50B1DF
:108AE00002988188E18000882081BDF800100298FA
:108AF00005F070FBDCE70A20DAE70A4B6A46002142
:108B0000A01D05F0A5FA38B1064918398E61CE616D
:108B10000A28CDD12846CBE702488188019805F084
:108B200059FBF5E7282300202DE9F0470025DFF861
:108B30008C803CE06068002100EBC50601203278A3
:108B40009146FDF780FCD4E9062300EA020701EA1A
:108B5000030C57EA0C0728D082438B434846C4E9EC
:108B6000062303F077FD32788246914601200021EA
:108B7000FDF769FCD4E9042300EA020401EA0307D3
:108B80004A4650460021FDF75EFC44404F403C43BE
:108B90000BD17078012801D0012100E0002172681A
:108BA00081EA0A010AB1484690476D1CEDB298F877
:108BB000000044468542BDD3BDE8F087C8220020AE
:108BC00010B50021024801F091FE80F3100010BDA5
:108BD000B03100200E4910B50A784C780023A2422B
:108BE00012D0521CD2B20A70022A00D10B70084A6D
:108BF0000B780C3252F8232002608868104420F071
:108C00007F408860012010BD0360002010BD00007F
:108C1000E822002013460A460021FFF785BE000027
:108C20002DE9F843104D0F4680461E469146694691
:108C3000286801F0B6FD040014D01C21FDF72FFCBC
:108C400001202071C4F81490380BC4F80080C4E9E6
:108C500002606946286801F0C5FD05F08DF9002025
:108C6000BDE8F8830420FBE7B0FB020010B50378F1
:108C70000022072B06D2DFE803F0050406102029A6
:108C800030000A7010BD01230B7003898B8183882B
:108C9000CB81C06888600A7410BD02220A70028904
:108CA0008A818288CA81C2688A60807D062802D053
:108CB0000020087410BD0120FBE703220A70C2885F
:108CC0008A810289CA81C068886010BD04230B7044
:108CD000C0888881CA818A6010BD0520087010BDD7
:108CE00070B5064D0646002455F8241009B13046EB
:108CF0008847641C042CF7D370BD0000F42A0020C0
:108D000030B50446006887B00D46806800281FD043
:108D100018216846FDF7C3FB0195A06805902079EE
:108D200010B1012810D107E001208DF80000206962
:108D30000290E068039005E002208DF80000E068F2
:108D40000003029060690490206881686846884743
:108D500007B030BD70B586B015460C00064619D078
:108D6000112C17D0082C15D014216846FDF797FB5D
:108D7000ADF80260304600F01FFFADF804000D2C86
:108D80000AD0862C1CD007208DF80000029468467B
:108D900000F04CF806B070BD03208DF8000025B13E
:108DA0002878C00701D0012000E002208DF80800DB
:108DB00000208DF80C0041F20110ADF80A00E6E742
:108DC00006208DF80000E2E710B50446408800F068
:108DD000F3FEA080024801682046BDE81040084725
:108DE000502200202DE9F04107460024064E074D91
:108DF00005E000BF56F8241038468847641CE87820
:108E00008442F7DBBDE8F08150280020702200206A
:108E100010B50446408800F0CFFEA08002480168EB
:108E20002046BDE8104008479CFA02000149096845
:108E300008470000F0FA020070B586B0044614211D
:108E40006846FDF72CFBA0890125A0F54040ADF850
:108E5000040020782A4E062833D2DFE800F03203DF
:108E600003032C48A08900F0BDF930B9E08943F62E
:108E7000FE71A0F54040884223D8A07B8DF8080001
:108E8000207803280FD000208DF80900A0680390F7
:108E9000606850B109208DF8000060680490684651
:108EA00004F0ECF90DE00120EEE708208DF8000059
:108EB0008DF81050F3E7A08900F094F908B1E0892B
:108EC00030B17078002801D004F008FB06B070BD06
:108ED000606820B10B208DF800007570DFE70A2074
:108EE0008DF80000BDF8040004F082FBF5E71320C4
:108EF0008DF800004FF6FF70ADF80400CFE70000DA
:108F00006022002038B504460E480078A8B1A4F5C8
:108F10007F40FF380FD0684604F060FF78B105212C
:108F2000017001210171C480684604F065FF05F0FD
:108F300015F8002038BD042038BD022038BD0820B7
:108F400038BD0000302300200C4808B5007888B1F7
:108F5000684604F043FF78B106210170684604F0CA
:108F60004BFF0748017809B10121017304F0F6FFB6
:108F7000002008BD022008BD082008BD30230020C5
:108F8000B82B0020F0B587B014216846FDF787FAAA
:108F90002B4C207818B16846FFF7A2FE4EE0201D4A
:108FA00001F086FCB8BB4FF0102041690004026953
:108FB00040694B1C01D100FB02F1224800220161F3
:108FC000A1F54051C160204902F0F8F8002820D1F5
:108FD0001F481C238C221D49006801F0CFFB03F0C1
:108FE0003DFF051E14D0022812D000270126062DB1
:108FF00012D005A804F0F2FE88B106700C2D18D22C
:10900000DFE805F0170F170F1716171617111311B2
:109010000B2007B0F0BD11E026706760BBE70820A9
:10902000F7E7077105E0032100E00221017100E08C
:10903000067105A804F0E0FE04F090FF0020E8E7C8
:1090400030230020E0230020C0FB0200042B00207E
:1090500028FB020038B5040014D0694605F03CF83E
:10906000A0B1BDF8000000EB8001094800EB8100D1
:10907000C16849B1A17A39B1C168491EC1600020F7
:10908000A07238BD052038BD062038BD0A2038BD85
:10909000902B00201FB501A9684604F0D9FF04B049
:1090A00010BD07B513460A466946002004F0D0FFFC
:1090B0000EBD07B513460A460021684604F0C8FFF6
:1090C0000EBD20B119B1006808600020704705206E
:1090D00070470000F8B50D46040018D0BDB16946D0
:1090E00004F0FAFFA8B1BDF800000B4900EB8000C6
:1090F00001EB800001210C30666801F0DCFB2E6082
:1091000060680C3068600120A0720020F8BD052066
:10911000F8BD0A20F8BD0000902B002018B10323F1
:10912000002206F019BB052070470223002206F03A
:1091300013BB12B1022306F00FBB052070470000DD
:10914000084910B50A69042A0AD0074A096942F891
:10915000210004480121103001F0ADFB002010BDBA
:109160000C2010BD10230020F42A002038B504463E
:1091700009480D46007858B164B16946284606F0A2
:10918000E5FB002803D1BDF800102180658038BDC3
:10919000022038BD052038BD3023002010B504461C
:1091A0000E48007898B1A4B12188022913D80C4A3E
:1091B00001EB810002EB800260885289C31C93425C
:1091C00009D806F0B7FB00202080608010BD022087
:1091D00010BD052010BD042010BD0000302300206C
:1091E000902B002043F6FE71A0F54040884201D844
:1091F000012070470020704710B5044600781828F9
:1092000002D1FEF795FA207010BD10B50446007823
:10921000182802D1FEF78CFA207010BD70B50D46EB
:109220000446B0F89810D0F894000122FDF7EBFF47
:1092300000B1057004F13C0204F1940104F1540002
:1092400072DF70BD70B513460022064615468629AA
:1092500002D0112902D002E0012200E001250D4CCC
:1092600073B1A179FEF788FA2A4661793046FEF794
:1092700083FA0022A1783046FEF77EFA002203E04E
:10928000A178FEF779FA2A4661783046BDE8704049
:10929000FEF772BA88220020F7B517460E0011D0EB
:1092A0000098002560B100242146684601F0E5FAE7
:1092B00018B1A0B23946B0476D1C641C142CF3D30E
:1092C0002846FEBD0020FEBD406804F0A7BD00009A
:1092D00070B508B1012070BD194C0025207B08B184
:1092E000257301E000F0A0F82078082826D2DFE8F6
:1092F00000F02504080C10251420BDE8704000F093
:1093000021B8BDE8704000F07DB8BDE8704000F0C5
:109310005FB8BDE8704000F03BB86088084900EBDA
:109320008000283901EB80004068BDE8704003F000
:1093300075BD6560BDE8704003F07EBD0F2070BD57
:10934000B82B00201149F0B48A1C00200346A1F17B
:1093500028050C18A67A4EB1A37200EB800405EB29
:109360008404E66816B9247C012C0AD0401C80B223
:109370000228EED30B704B804B60F0BC41F61D50C1
:1093800070471080F0BC00F03DB80000B82B002002
:109390000C48418801EB8102A0F1280101EB820118
:1093A000CA6852B105210170074802218180016815
:1093B00000230122054801F06BBE042202704968B7
:1093C000F6E70000B82B002038230020E02300201F
:1093D00038B50A49084803240B684268898803EBBA
:1093E000810153880470DB1C00201B0400909B0B40
:1093F000034801F0BDFF38BDB82B00203823002002
:10940000E0230020074910B54888091D04F0B4FE88
:1094100018B1BDE81040FFF7DBBFBDE81040FFF713
:10942000B7BF0000B82B0020F0B51F481F49012529
:10943000067802248B88A0F12802082E19D2DFE8D2
:1094400006F00418181B222F2F170189491C0181CF
:109450000021418080F80C1001EB810312F82330C9
:1094600043B100234418491C89B2A3720229F3D3E3
:109470000570F0BD0123F5E742685288D21C1A44FA
:109480008A800470F0BD46880D6806EB860602EB04
:10949000860256680E60556013818C80062100E0BC
:1094A00007210170F0BD0000B82B002038230020F8
:1094B00030B501888488224D85B0502924D05229A6
:1094C00002D0542931D103E0204600F07FFE2CE089
:1094D00014221C496846FCF7C9FFADF8024020463B
:1094E00000F06AFBADF8040000F022F9002269796F
:1094F0002046FEF741F9002229792046FEF73CF983
:109500006846FFF761FC10E0017B01290DD1817AEB
:1095100001290AD10089A0F52451023905D1012180
:10952000204600F087FE05F03DFF00220649E8785E
:10953000FEF7D6F805B0BDE8304005F09DB8000054
:109540004822002018FA0200B16F020010B504464C
:10955000007800280FD1608800F038FE608800F0A5
:1095600081F9002807D00449608801220979BDE803
:109570001040FEF701B910BD4822002010B5124C72
:1095800000202070FEF7D4F8A070FEF7D1F8E0704C
:10959000FEF7CEF82071FEF7CBF86071A17818299C
:1095A0000FD0E17818290CD02179182909D0182872
:1095B00007D00121601C04F0F7F901202070002081
:1095C00010BD032010BD0000482200207CB50446D9
:1095D000007808282FD1607A38BB207A4FF6FF75C3
:1095E00001280DD0072802D0082824D11EE0A08829
:1095F00000F020FAA8421ED0012100F01BFE1AE064
:10960000A0886A46012103F051FD70B901980078E5
:1096100058B1A08800F00EFAA8420CD008490122E7
:109620000979FEF7A9F805F027F804E004480021BD
:10963000401C04F0F4F9BDE87C4005F0B3BE000026
:109640004822002010B504460A4841782046FEF71B
:109650007BF868B10848002101EB410200EB82026F
:109660005288A24201D1C8B210BD491C1429F3D3BB
:10967000FF2010BD5A2200204026002070B5094D61
:10968000094E002404EB440005EB8000717840880B
:10969000FEF75AF820B1641C142CF3D3FF2070BDE0
:1096A000E0B270BD402600205A2200202DE9F04192
:1096B0008046024601200021FCF7C5FE1A4F0546F0
:1096C0000E467868FDF7B0FB00280CD1174CD4E9A2
:1096D000062110462A4001EA06031A4305D0A84392
:1096E000B143C4E90601BDE8F081404602F0B2FF93
:1096F00030B1D4E9040128433143C4E9040105E051
:10970000D4E90410A943B043C4E90410D4E9060124
:1097100028433143C4E90601A1687868BDE8F041F7
:109720000022FDF73DBB000014FB0200C822002010
:109730001CB5054AD2E90212CDE9001200226946A1
:1097400003F0D9FC1CBD000030FA020003484FF6BC
:10975000FF71818001210170002070475422002098
:109760002DE9FC41804600F027FA0024032501275B
:10977000A0F57F412646FF3908D06A46082103F04C
:1097800095FC18B90198841D8688056832462B46D9
:1097900021464046B1DF042804D0082804D00B2815
:1097A00008D002E0112000E00020002F00D10B20A3
:1097B000BDE8FC810027A80701D50125E6E7344371
:1097C000F5D0002426460325E0E72DE9FC4180463C
:1097D00000F0F2F90646A0F57F40FF380ED00125D3
:1097E0002A466D1C0027ADB26B460821304603F0B7
:1097F00087FC040006D0072C25D025E043F20200A8
:10980000BDE8FC81019903230A1D0B604046891DB8
:10981000B2DF040004D00C2C09D0052C09D009E0DB
:1098200032460821104603F0E1FC04460CE0012713
:1098300000E000240821304603F0C4FC00B10324FA
:10984000002FCDD100E00C242046D9E704488088C1
:10985000A0F57F41FF3901D004F018BF7047000028
:10986000542200200EB502A9019100F0A5F96A4624
:10987000012103F01BFC08B100200EBD0198007807
:109880000EBD00002DE9F04107464FF6FF760A486D
:10989000B3DF10B10320BDE8F081074C43F20305AC
:1098A000A41E324661883846AFDFA842F3D16088F3
:1098B000401C6080F5E7000056220020428800EB43
:1098C00082020C328A4201D9022070478188A1F5B8
:1098D0007F42FF3A03D0008808B100207047012082
:1098E0007047884204D20068401C01D001207047B4
:1098F000002070473EB5027802230C46B3EB520FAE
:1099000017D1B0F80110ADF80010C1788DF8021031
:109910008188ADF8041080798DF8060002AA01A9AB
:109920002046FDF7F1F8032202A96846FCF7C9FDBD
:1099300008B100203EBD01203EBD000010B50C4620
:10994000FFF780FEFF280CD0074900EB400001EB39
:109950008000416821600189A180807AA071002087
:1099600010BD052010BD00004026002070B5018804
:1099700090B0102959D1011D2C226846FCF776FDC4
:109980009DF804004FF6FF76032134466D46B1EB97
:10999000500F2AD003F0E0FC9DF8040040080ED0E0
:1099A00001280CD0022820D118E00D99281D113172
:1099B000FDF746F818B100BFBDF82C4015E00CAA21
:1099C0000BA9072003F09CFC0028EED10DE00D99B7
:1099D000281D491CFFF78EFF0028EDD10CAA0BA90A
:1099E000072003F08DFC0028F1D1BDF80000291DEF
:1099F00000F06EFEB44218D0BDF80000214600F021
:109A0000C5F8BDF80000ADF82E000020ADF83040DC
:109A1000074E8DF82C000BAD044600BF56F82410FD
:109A200028468847641C022CF8D310B070BD000093
:109A300044FA0200094A002101EB410332F82330C5
:109A4000834205D101EB410002EB80004088704762
:109A5000491C1429F0D34FF6FF70704740260020B0
:109A60003EB50C46054603F077FC0BE0BDF8000060
:109A7000A04207D02846029900F02EF810B1BDF898
:109A800000003EBD01AA6946072003F039FC00280A
:109A9000ECD14FF6FF703EBD10B50D4C18200D4AAD
:109AA000607000204FF6FF7100EB400302EB830370
:109AB000401C59801428F7D3FDF73AFE607018282F
:109AC00003D001202070002010BD032010BD000035
:109AD0005A220020402600202DE9F0410C46054680
:109AE00000F1110701F111061022491C401CFCF77E
:109AF000E8FC48B9681C00F0F9F928B1601C00F0D6
:109B0000F5F908B1012400E0002431463846FCF79D
:109B100097FF3B780222B2EB530F0CD00321B1EB3D
:109B2000530F08D03378B2EB530F04D0B1EB530F7F
:109B300001D0012100E00021084201D18C4302D074
:109B40000120BDE8F0810020FBE7018811B942182F
:109B500092780AB101207047491C0829F7D30020E8
:109B6000704710B50C460346FFF7EFFF00280AD0F8
:109B700018882188884205D10822A11C981CFCF76E
:109B8000A0FC08B1002010BD012010BD03F084BD71
:109B900070B50446FFF74EFF0546204603F089FAEC
:109BA0004FF6FF7104468D4203D014B9284603F0E6
:109BB00073FD204670BD000010B5FFF743FDFF2880
:109BC00005D0044900EB400031F8200010BD4FF6ED
:109BD000FF7010BD402600203EB5044603F0BCFBDC
:109BE0000EE0019920464631FFF7BBFF28B90199E5
:109BF00020462A31FFF7B5FF10B1BDF808003EBD81
:109C00006A4602A9072003F07BFB0028E9D14FF642
:109C1000FF703EBD10B50A4941600A4800F048FE99
:109C200058B902F089FB07491C238C2208740448A8
:109C30008C39001F006800F0A1FD002010BD00005D
:109C4000B4FB0200542C00202DE9F0412D4F0025DB
:109C500018B17D600120BDE8F0810879012258B17A
:109C6000294E01280CD0274C4FF002080834022856
:109C700021D0032842D128E00A7103F0DDF83BE04F
:109C80005FF0000000EB800116F82110022908D0D7
:109C9000401C80B20228F5D33A707D6041F61D5019
:109CA000D9E700EB800006F8205006EB8000406802
:109CB00003F0B4F820E00D71A4F804800023012221
:109CC0001248216801F0E4F916E00D71206803F0F4
:109CD000A5F80D4923682831498801EB810206EB7C
:109CE0008201D1F804C0C4F800C04B60A3880B8186
:109CF000A4F8048006F822500028ACD07D600E2025
:109D0000A9E7000030230020902B0020E023002052
:109D10000146034802888A4200D0002070470000B4
:109D2000982500202DE9FC5F0E008346DDE90C47F5
:109D3000C6F1000098469246814600D408460125A7
:109D400003E000BF90FBFAF06D1C5045FADAA8451D
:109D500000D9454624B1002E01DB780700D5641EEA
:109D6000B80702D5B8F1000F0AD0F80708D13CB106
:109D7000A54205D220215846641EFEF753FCF6E7A3
:109D8000002E02DA4E462D2102E0780703D52B2162
:109D90005846FEF747FC07F0030002280BD1B8F144
:109DA000000F08D13CB1A54205D230215846641EAF
:109DB000FEF738FCF6E7CDE9004743465246314608
:109DC000584605F095FABDE8FC9F000070B50D46B9
:109DD000044600684FF4887102F044FB4FF4907120
:109DE000206802F03FFB4FF49271206802F03AFBCA
:109DF0004FF4A271206802F035FB20681249C0F8C8
:109E0000041320686907000B40B2090E002806DA27
:109E100000F00F0000F1E02080F8141D03E000F1D5
:109E2000E02080F8001420680121000B40B200F00F
:109E30001F0291404009800000F1E020C0F880122C
:109E4000C0F8001170BD000010030200024600209F
:109E50001268930702D0530702D47047500714D5F5
:109E600002F00300012802D002280CD105E0C2F361
:109E700083100B68801C184404E00223086803EB7D
:109E800092521044086001207047086800EB92531A
:109E9000C2F38910401CEEE70248007A002800D087
:109EA00001207047542C0020F0B58488A5189442F6
:109EB00000D82246A41AC288D6189A4200D813465F
:109EC000D21A4B880788BB420CD34088834209D8FA
:109ED0008888A04206D3A84204D8C888904201D3FB
:109EE000B04201D90020F0BD0120F0BD0021425C4C
:109EF0000AB101207047491C1029F8D3002070478F
:109F0000800701D000207047012070470A4810B533
:109F1000807860B1002401E0022C06D02046FEF7D4
:109F2000F9F8641C042CF7D310BD0324F6E7BDE850
:109F30001040FEF713B900002822002003480179E1
:109F4000C90702D00078FEF745BA704728220020E2
:109F50001721018041800021017141711B21817114
:109F6000C17170472DE9FE4F2B4D984691460F0069
:109F7000824601D000260DE0684600F0D5FB6A4617
:109F80000021504603F001F82878009E10B99DF892
:109F9000090098B14A463146504604F0D3FD0446C4
:109FA000014600225046FFF74DF90D2C32D008DC57
:109FB00084B3082C2ED00B2C0BD12BE00520BDE850
:109FC000FE8F112C10D0862C1AD0A4F540500238E8
:109FD00020D00325B8F1000F04D032462146504668
:109FE000FEF7B8FE2846EAE73A4629795046FDF7DB
:109FF000C3FB4A46E9785046FDF7BEFB0025E9E77A
:10A000003A4629795046FDF7B7FB4A46E97850466B
:10A01000FDF7B2FB2546DDE7882200202DE9F0415F
:10A02000204F0E46154604463978FDF78DFB002873
:10A0300035D0204602F0A0FF50B32046FFF7BCFD0C
:10A0400080462046B978FDF77FFB08B1012700E084
:10A050000227204603F038FA0028404602D0FFF7D6
:10A0600097FD0DE0A8F57F41FF3909D0072103F0E6
:10A07000A9F8010004D0052902D0204604F0C8FA4E
:10A080002B46324639462046BDE8F041FEF74CBC2F
:10A090002A4631462046BDE8F041FEF7BBBDBDE88B
:10A0A000F08100008022002070B5094D0646E97855
:10A0B000FDF74AFB044629793046FDF745FB01468A
:10A0C00022463046BDE870400123FFF74BBF000039
:10A0D000882200202DE9F047394E002780463D4672
:10A0E000DFF8E090D6F804A057E003D00446D0F89B
:10A0F0001C8035E099F8002002EB4201521CD2B2DC
:10A1000089F8002009EBC10199F80230091D9A4233
:10A1100001D189F8005048680A780446012A12D013
:10A12000022A02D0032A3BD108E004F0B3FE00B1BA
:10A130000127257434E00574C06900E070680028C8
:10A14000F9D170602CE0207C50BB88686060C868E2
:10A15000A0600869E0604869A061F07800B16560BE
:10A160006268B168184B501A20F07F40984202D2C2
:10A17000A168084406E0881AA16820F07F40814267
:10A1800002D9081A206000E0256065600120A56002
:10A1900020742046E56104F05FFEB8F10000A4D110
:10A1A00099F8001099F801008142A3D117B971689C
:10A1B000514502D00120BDE8F0870020FBE70000F8
:10A1C000E8220020D0290020FFFF7F0030B585B0B5
:10A1D0000546002414216846FCF761F9A5F57F4087
:10A1E000ADF80250FF3815D02846FFF7B9FA98B1FC
:10A1F0000B2815D0112811D0A0F54051023903D0F9
:10A200000146284604F0F0F909482246C17828465C
:10A21000FDF7B2FA05B030BD0E2002E00124F3E7ED
:10A220000F208DF800006846FEF7CEFDECE7000039
:10A23000482200200A4602498978FDF79DBA0000AD
:10A2400048220020F8B5054600780C46002620423A
:10A250000FD100208DF800006846FCF7F5FD287846
:10A26000204202D12043287001269DF80000FCF70F
:10A270000FFE3046F8BD00002DE9FF4100262348BF
:10A2800000F013FB2148001F074600F00EFB204C96
:10A2900060680090A56800E000986946284004EBDB
:10A2A00080000C30FFF7D2FD0028F5D101AA0099FB
:10A2B00001EA050304EB8303491CDB6842F8203004
:10A2C000401C00910228F2D3019800F003000128FD
:10A2D0000BD0022810D10198032101EB9050009976
:10A2E000BDF80A6001EB900005E00198BDF80A6036
:10A2F000C0F3831008440090384600F0D3FA08B148
:10A300000098606004B03046BDE8F081AC310020B8
:10A31000942D0020ACB04FF40041002001F0B2FCBD
:10A3200008B1FCF7AFFC01F01DFBFCF70FFD08B115
:10A33000FCF7A8FC01F0C4FD08B1FCF7A3FC6349DD
:10A340000320FDF7FDFF08B1FCF79CFC69460020E7
:10A35000FDF728FF08B1FCF795FC9DF800000228E6
:10A360007DD0002501F09CFF08B1FCF78BFC002498
:10A3700069460120009401F021FE08B1FCF782FC3F
:10A38000684601F09FFE08B1FCF77CFC03F092F9EF
:10A390009DF808004EA120F00F00401C20F0F000B6
:10A3A00010308DF80800112202A87CDF08B1FCF7FC
:10A3B00069FC00945020ADF80000A0200194ADF895
:10A3C0000200ADF804404FF4C870ADF806006846CE
:10A3D0007ADF08B1FCF756FC0021424800F0FBFA96
:10A3E00008B1FCF74FFCAC216846FCF758F8022096
:10A3F0008DF8000001208DF802000621ADF8100054
:10A400008DF87C008DF803104FF496703649229039
:10A41000059144F2506023903448299031486946B0
:10A420002030FCF71FFF08B1FCF72CFC2D48012160
:10A430002030FCF714FF2E4801A9CDE9004029483F
:10A44000143000F088FB08B1FCF71CFCFDF7EEF9B6
:10A4500008B1FCF717FC27480090684600E032E09E
:10A46000FDF790FA08B1FCF70DFC1C216846FCF7DB
:10A4700016F84FF42030CDE900404FF470200290E0
:10A480001D48059003261D488DF80C600690ADF818
:10A490000E408DF810406846FDF7DEF808B1FCF775
:10A4A000F1FB174817A1008806EB004001F078FB8C
:10A4B0002846FCF705FB00BF01F062FA0028FBD13B
:10A4C00001F026FDF8E701254CE700009982020023
:10A4D0004E6F726469635F427574746F6E6C6573FE
:10A4E0007300000034240020222200207DCB0200D3
:10A4F000A5BF0200257C0200A1CB0200DB88020080
:10A5000024240020427574746F6E6C65737320444C
:10A510004655204170706C69636174696F6E207379
:10A520007461727465642E0070B5144682880E469C
:10A5300005462088111D0144921C994201D8FE2A2B
:10A5400001D90C2070BD521C32542088FF21401CC0
:10A5500080B2208031542088401C80B22080811934
:10A56000288804F0AFFE2188084480B22080AA88A1
:10A5700042B1A96841B13044FBF778FF2088A9882F
:10A5800008442080002070BD072070BD2DE9F047F1
:10A59000C7880446181D16468946B0FBF7F1B0FB84
:10A5A000F7F207FB12009A193A44D21CB2FBF7F2F9
:10A5B000DDF820A001E02468491E0029FBD13D1AE6
:10A5C0008846B54216D818E0BAF1000F05D0211818
:10A5D00009EB08002A46091D04E0204409EB0801A4
:10A5E0002A46001DFBF742FF00202468761BA84482
:10A5F000B74201D9354600E03D46002EE4D1BDE822
:10A60000F087000030B5024659B101F067FB002128
:10A61000074C09E004EB810315685B88AB4202D16B
:10A620001160002030BD491C8142F3D3052030BDAC
:10A63000F4230020F8B50F46017814460546012999
:10A6400001D1687830B12088821C9A422DD8012926
:10A6500002D006E00720F8BD69780144891C9942C0
:10A6600023D8181A801E86B2ADF800602188B81C65
:10A67000084469467DDF0028EDD12878022805D1FD
:10A68000BDF80010B14201D809210AE008210128D3
:10A6900005D16878B04202D8ADF8000001E0ADF80D
:10A6A0000060BDF80000FE2801D90C20F8BD22880A
:10A6B000401CB8542088401C80B220803954208827
:10A6C000401C2080BDF80010084420800020F8BD08
:10A6D00070B505460C004FF0FF0020D04FF6FF7616
:10A6E000B5421CD00E48012241782846FDF744F8B7
:10A6F0002846FEF7A7FFFF2803D1FEF7BFFFFF287C
:10A700000DD0084B00EB400203EB82014D8023F893
:10A71000226022684A60A2880A81A2798A7270BD8A
:10A720005A22002040260020034A00219268C0E9F6
:10A7300000218160704700008822002070B54FF62C
:10A74000FF750E46A84201D1002000E0401C84B2F3
:10A7500008E02146304603F056F908B1204670BDA6
:10A76000641CA4B2FF2CF4D9284670BD10B5FBF7C9
:10A770009CFD08B1002010BD112010BD10B531B1F5
:10A78000B2FBF3F403FB14241CB1092010BD0E200E
:10A7900010BD01600021416081608281C381084653
:10A7A00010BD70B50C460546FBF734FD002802D0FD
:10A7B00021882868084470BD10B50A8849888A42F3
:10A7C00003D1FBF769FD012010BD002010BD70B55D
:10A7D0000C460546FBF743FD002802D06188286837
:10A7E000084470BD10B50A8849888A4203D1FBF736
:10A7F0002DFD012010BD002010BD01F01F0301221E
:10A800009A40D243490900EB8100114600F059B843
:10A810000A4601F01F030121994010B552090C4668
:10A8200000EB820000F05DF8204000D0012010BD58
:10A830002DE9F04180460D460024481E012101EB20
:10A84000501716E058F82400C04390FAA0F0B0FA70
:10A8500080F020280CD200EB4416AE4208D23146DC
:10A860004046FFF7D5FF0028ECD13046BDE8F08127
:10A87000641CA742E6D82846F8E74A0950F82200A7
:10A8800001F01F0201219140084000D001207047D3
:10A8900001F01F0301229A40490900EB8100114693
:10A8A00000F029B8002100F017B8012100F023B80A
:10A8B000012100F016B808B56A46FBF742FD009882
:10A8C00008BD08B56A46FBF722FD009808BD08B52B
:10A8D0006A46FBF736FD08BD08B56A46FBF717FD6B
:10A8E00008BD08B56A46FBF705FD08BD08B56A4610
:10A8F000FBF7F4FC08BD08B56A46FBF7FBFC0098C3
:10A9000008BD08B56A46FBF729FD009808BD38B5B3
:10A91000044600258DF800506846FCF795FA21683A
:10A920006268086890420ED9401E08600178A38AC8
:10A93000E26801FB0325227A2168101AC0B20A7965
:10A94000824200D208719DF80000FCF7A1FA284667
:10A9500038BD38B5054600208DF800000C46684625
:10A96000FCF772FAE868A98A201AB0FBF1F12A68AC
:10A970001068431C136001709DF80000FCF788FA12
:10A9800038BD10B530B1017A42680368891AC9B27E
:10A990001A6006E00E2010BD03681A68541C1C6083
:10A9A0001170491EC9B2F7D2006800210171084632
:10A9B00010BDC20800F007030120895C98400840E0
:10A9C000704710B5C20800F00703885C01249C4062
:10A9D0002043885410BD10B560B10161172120F8E3
:10A9E000021B20F8021B1B2100F8021BFFF7B0FA24
:10A9F000002010BD0E2010BDF0B5858893B00C4628
:10AA0000002D39D1018800263E4F24293BD006DC99
:10AA1000102909D011290CD0232958D14FE03A2907
:10AA20000BD0552953D129E00146204602F0C6F843
:10AA30004DE0A01DFFF78CFA49E02246408934F82A
:10AA4000061F814200D808466080172800D21720D0
:10AA50006080106970B1607960B1D7E90001CDE91B
:10AA60000301ADF80E506088ADF81000136903A91A
:10AA7000104698476671267113B0F0BD0146204616
:10AA800002F0ECF823E0011D2C2206A8FBF7EEFCF7
:10AA9000BDF81800BDF81C2004EBC0014A73226900
:10AAA000AAB1D7E90423CDE90423ADF81200487B0D
:10AAB0008DF814002269204604A9904707E0017A26
:10AAC000207B884200D201462846FDF74FFFA07A3E
:10AAD0000028D1D0E1882846A5DF012570B11128D2
:10AAE000CAD001F09FFC0246074808A1008813B0B5
:10AAF00005EB0040BDE8F04001F056B8A672E572E3
:10AB0000BAE700004CFA0200F423002073645F628D
:10AB10006C655F67617474635F65786368616E67B5
:10AB2000655F6D74755F7265717565737428292032
:10AB300072657475726E65642025732E00000000C6
:10AB400020B10278DE2A03D0082070470E2070471B
:10AB500041800020704760B159B10278DE2A0AD0E6
:10AB600009684160DE2101704FF6FF7141800020CD
:10AB700070470E207047082070477FB505460029B2
:10AB80004DD0002D4BD008780C46DE2847D1A88840
:10AB90006188884202D1204604F054FC28880128AC
:10ABA00025D002283BD011283AD0512837D135F88A
:10ABB000040F6188884232D1A978A81C02292ED1BD
:10ABC000017A042903D0062901D0052927D10021C3
:10ABD000009102228DF8002001914FF4C072029181
:10ABE0000391ADF80420007A05280FD010E0297AEF
:10ABF0002046012913D1A988428891420FD1012111
:10AC0000017204B0BDE8704004F01CBCADF8041043
:10AC100028886946B0DF002801D0616888477FBD79
:10AC2000A88861888842FAD14FF6FF7060807FBDA6
:10AC300000F180400068002800D00120704708B56E
:10AC400000F18040002101600068009008BD000014
:10AC500070B54FF010246169104D0126491C2888F9
:10AC600014D06269032101EB00400DA100F09CFFAC
:10AC7000606913DF040007D0288814A106EB0040A8
:10AC800000F08EFF204670BD002070BD06EB004036
:10AC90001BA100F085FF042070BD000024240020CB
:10ACA00053657474696E6720766563746F7220747F
:10ACB00061626C6520746F20626F6F746C6F616489
:10ACC00065723A2030782530387800004661696C2A
:10ACD00065642072756E6E696E672073645F736F52
:10ACE00066746465766963655F766563746F725FC9
:10ACF0007461626C655F626173655F7365740000A7
:10AD00004E6F20626F6F746C6F6164657220776143
:10AD10007320666F756E640070B50C4D03210C4A8C
:10AD2000288801EB00400BA100F03EFF084813DF2C
:10AD3000040008D02888012101EB004010A100F098
:10AD40002FFF204670BD002070BD0000242400208D
:10AD50000060020053657474696E672076656374E1
:10AD60006F72207461626C6520746F206D61696E12
:10AD7000206170703A20307825303878000000006B
:10AD80004661696C65642072756E6E696E672073CA
:10AD9000645F736F66746465766963655F76656327
:10ADA000746F725F7461626C655F626173655F731B
:10ADB0006574000070B50B4C207808B185250FE054
:10ADC0000020A06060602061E060074801F066FB41
:10ADD000054601F0B1FA08B901F04AFB01202070E4
:10ADE000284670BDE02800204D87020038B50025B8
:10ADF0008DF800506846FCF727F8074CE068401EC5
:10AE0000E060E06810B901F059FBA5709DF8000002
:10AE1000FCF73EF838BD0000E0280020F0B50546FC
:10AE20000478154889B0164640F82420124A08696B
:10AE30000832A2F10C0742F82400487F385520223E
:10AE40006846FBF713FB04942878385C48B10EB1D0
:10AE50000A4A00E000226946281D01F0ABFD09B056
:10AE6000F0BD0EB1064A00E00022694605F10C0073
:10AE700001F072FCF3E70000A8220020A1F102001B
:10AE8000EDEF02000FB408B50399002904D004AA1D
:10AE900000926A4600F00FF801B05DF814FB10B59F
:10AEA00082680446002A05D0D4E904032168984743
:10AEB0000020A06010BD2DE9FC4791460C008046A3
:10AEC00076D014F8011B39B125290ED04046FDF784
:10AED000A9FB20780028F4D198F80C00002867D04E
:10AEE0004046BDE8FC47FFF7DABF00200122217889
:10AEF0002B291BD02D2902D0302908D102E040F0A7
:10AF0000010001E040F00200641C002AEFD100259E
:10AF10002A290ED02178A1F130020A2A11D205EB9C
:10AF2000850201EB4205641C303DF1E740F004006E
:10AF3000EAE7D9F800100B1DC9F800300968641C55
:10AF40000D44217800232E290BD114F8011FA1F103
:10AF500030020A2A05D203EB830201EB4203303BA5
:10AF6000F3E76C290DD068290BD0692921D00BDCBF
:10AF7000252918D0582931D063290ED0642915D13C
:10AF800017E014F8011FECE7702969D0732932D05B
:10AF900075291BD0782909D120E0D9F80000011DBE
:10AFA000C9F8001001784046FDF73CFB641C90E7AF
:10AFB0006CE0D9F800100A1DC9F800200968CDE935
:10AFC00000500A224046FEF7ADFEEFE7D9F8001028
:10AFD0000A1DC9F8002009680A2206E0D9F8001005
:10AFE0000A1DC9F8002009681022CDE9005040462A
:10AFF00004F07EF9DAE7D9F8001000270A1DC9F835
:10B0000000200E68C00705D112E04046761C7F1C68
:10B01000FDF708FB31780029F7D104E020214046F4
:10B020006D1EFDF7FFFABD42C0D9002DF6D1BDE778
:10B030004EB13046FBF73EFA074604E02021404679
:10B040006D1EFDF7EFFABD4206D9002DF6D103E0E3
:10B050004046761CFDF7E6FA31780029F8D1A5E7DD
:10B06000D9F80000011DC9F80010056830214046DC
:10B07000FDF7D8FA78214046FDF7D4FA08200021E0
:10B08000CDE90001034610222946B0E7BDE8FC8760
:10B090002DE9F84F2B4E04009A4630884FF00103FB
:10B0A0001546894603EB004024D0216800292BD0A7
:10B0B000002D32D0626849464FF010071268A2F1A5
:10B0C000010C1CEA090F11D198466A432046FBF790
:10B0D000D0FC00282AD0206853462A46066901B0D1
:10B0E00049462046B446BDE8F04F6047164B17A2CC
:10B0F000009721E00E210091134B1EA21FA100F02A
:10B1000062FD0E20BDE8F88F082100910E4B26A2AB
:10B110001AA100F058FD0820F4E7092100910A4B1C
:10B1200024A216A100F04FFD0920EBE7009731881B
:10B13000054B214A08EB014010A100F044FD10200E
:10B14000E0E70000142400209BFB020061646472AD
:10B150005F69735F706167655F616C69676E656485
:10B1600028705F66732C20706167655F616464722C
:10B1700029000000705F66730000000025732063E3
:10B180006865636B206661696C656420696E202563
:10B1900073282920776974682076616C7565203082
:10B1A0007825782E00000000705F66732D3E705F7A
:10B1B000617069006C656E001000030038B5030013
:10B1C0000F484FF001054FF00E04008805EB0040DA
:10B1D00009D061B119600C6801B0A446BDE83040E7
:10B1E000114618466047074B07A2009402E0054B42
:10B1F00007A2009408A100F0E6FC0E2038BD000074
:10B200001424002050FB0200705F667300000000F1
:10B21000705F617069000000257320636865636B6F
:10B22000206661696C656420696E20257328292079
:10B23000776974682076616C756520307825782E82
:10B24000000000002DE9F04128B1016819B1C96979
:10B25000BDE8F04108470D4D0D480024461B14275A
:10B260000DE000BF04EB840005EB8000016829B10C
:10B27000C969884710B10120BDE8F081641CB6FBA4
:10B28000F7F0A042EED80020F6E70000E02300200F
:10B29000F4230020044801214174007A08B1002001
:10B2A0007047012070470000542C0020012801D075
:10B2B000032808D10449002201284A7400D0002044
:10B2C000087402F0FBBD7047542C002070B5024694
:10B2D000022801D0032A45D1234C207A002841D0EE
:10B2E000012833D0022831D120480023022A0068E7
:10B2F00002D0032A2AD11BE0E360017911B10129B0
:10B3000024D10DE0D0E90565711B4FF48056B142A0
:10B3100000D33146294481614569A9420ED015E028
:10B320000169491C0161426991420FD1237213E006
:10B33000E168491CE160082908D9E3602372022A08
:10B340000AD00D21FDF7DCFC02F05EFD607C28B127
:10B35000BDE8704000F0F6BF0021F3E7BDE87040A3
:10B3600002F0ACBD70BD0000542C0020542300201E
:10B370002DE9F84F3A4D04008B4628884FF001061E
:10B38000DDF828A0984691464FF00E0106EB0040EC
:10B390001AD0B9F1000F1BD02168002920D0092153
:10B3A000B8F1000F25D062685368B8FBF3F703FBD0
:10B3B0001782002A21D02B4B2BA2009135A100F03F
:10B3C00002FC0920BDE8F88F264B3DA2009102E067
:10B3D000244B3DA200912FA100F0F5FB0E20F1E7D8
:10B3E000082100911F4B3AA22AA100F0ECFB082093
:10B3F000E8E71C4B39A20091E0E75846FBF733FB26
:10B40000102798B14846FBF72EFBB0B1424659468B
:10B410002046FBF72EFBB8B1CDF800A020684346CC
:10B420004A46C56859462046A847CBE70097288872
:10B430000C4B06EB00402AA20CE000972888094B31
:10B4400006EB00402CA205E000972888054B06EB90
:10B45000004032A20FA100F0B6FB1020B2E70000BE
:10B460001424002088FB020021286C656E20252012
:10B47000705F66732D3E705F666C6173685F696EA6
:10B48000666F2D3E70726F6772616D5F756E697465
:10B4900029000000257320636865636B206661697D
:10B4A0006C656420696E202573282920776974688B
:10B4B0002076616C756520307825782E00000000BC
:10B4C000705F667300000000705F737263000000BD
:10B4D000705F66732D3E705F617069006C656E0011
:10B4E000616464725F69735F616C69676E65643320
:10B4F0003228646573742900616464725F69735FE4
:10B50000616C69676E65643332282875696E7433BF
:10B51000325F7429705F7372632900006164647222
:10B520005F69735F77697468696E5F626F756E6477
:10B530007328705F66732C20646573742C206C65AF
:10B540006E2900002DE9FF411C46DDE90A78154609
:10B550000E46684600F0AAF846EA450141EA840131
:10B5600041EA072242EA0841009A00EB8200C0F853
:10B570000017BDE8FF812DE9FF411C46DDE90A788F
:10B5800015460E46684600F09FF846EA450141EA36
:10B59000840141EA072242EA0841009A00EB820056
:10B5A000C0F80017BDE8FF812DE9FF411C46DDE929
:10B5B0000A7815460E46684600F094F846EA4501BA
:10B5C00041EA840141EA072242EA0841009A00EB7D
:10B5D0008200C0F80017BDE8FF812DE9FF411C463D
:10B5E000DDE90A7815460E46684600F089F846EA15
:10B5F000450141EA840141EA072242EA0841009AF2
:10B6000000EB8200C0F80017BDE8FF811CB50021E7
:10B6100000910B4601220191FFF7C6FF1CBD1CB52E
:10B62000002100910B4601220191FFF7D6FF1CBDBE
:10B630001CB500220B46009211460192FFF7B4FFA1
:10B640001CBD1CB500220B46009211460192FFF76B
:10B65000C4FF1CBD1CB5002100910B4601220191C5
:10B660001146FFF7A1FF1CBD1CB5002100910B4640
:10B67000012201911146FFF7B0FF1CBD13B50C4626
:10B68000684600F021F8009900EB8101D1F800270D
:10B6900022F44032C1F80027009900EB8100D0F875
:10B6A000001741EA0441C0F800171CBD01682029B9
:10B6B00002D24FF0A040704701F01F010160014825
:10B6C00070470000000300500168202902D24FF0AB
:10B6D000A040704701F01F01016001487047000061
:10B6E000000300500168202902D24FF0A0407047AB
:10B6F00001F01F0101600148704700000003005085
:10B700000168202902D24FF0A040704701F01F01CC
:10B7100001600148704700000003005001B5684611
:10B72000FFF7D2FFD0F810050099C84000F00100E3
:10B7300008BD01B56846FFF7D5FF009A0121914089
:10B74000C0F8081508BD01B56846FFF7D9FF009A93
:10B7500001219140C0F8081508BD38B501240090BA
:10B76000684631B1FFF7A2FF00998C40C0F8084548
:10B7700038BDFFF79BFF00998C40C0F80C4538BDE1
:10B780001CB5094C0144D4E90034CDE900346C46C1
:10B7900006E000BF54F82030D3F81035401C08C232
:10B7A0008142F7D81CBD000004FB0200034908B524
:10B7B0000844002101600068009008BD006000405E
:10B7C00002494058012800D0002070470060004026
:10B7D00030B5124B01460020D3F81044224609E050
:10B7E000157A854205D1401C0A28F7DB4FF0FF305F
:10B7F00030BD5268002AF3D1421CF9D00872D3F848
:10B8000010242AB152684A60D3F81024516030BD28
:10B810000022C3F810144A6030BD0000942D0020AF
:10B82000F0B595B01C4615460F4608461A9E00F026
:10B8300025FB182109A8FAF732FE0E96CDE9095426
:10B840000023082203A9384600F02DFB0598069036
:10B85000BDF81000ADF81C00BDF81200ADF81E00D8
:10B8600000208DF821000398082600F0030001282D
:10B8700002D0022818D032E003983346850AC0F37C
:10B88000C2008DF8200003980FA9C0F38314A20012
:10B89000384600F008FB09A8009006AB22460FA925
:10B8A000284600F047FA1AE00398840DC0F3C2005E
:10B8B0008DF82000082C01D2254600E008253346EB
:10B8C0002A460FA9384600F0EEFA2E44641B09AB55
:10B8D00006AA29460FA800F07FF9002CEAD13846C5
:10B8E00000F0D2FA15B0F0BD7047012003F09CBB08
:10B8F000084810B50178084A515C19B1001D01F0E3
:10B90000E5F802E00C3000F0F3FFBDE81040002045
:10B9100003F08ABB68230020A422002008B5034A54
:10B9200000924023024AFFF77BFF08BD39E6020080
:10B93000942C00200A4A012902EBC00007D00229FA
:10B9400007D0032907D0042907D000207047022020
:10B9500070470420704700797047407970470000B5
:10B960000C07030010B5FFF7C0FF04210348FFF7E1
:10B970002FFF02490120487210BD00007C230020E7
:10B980002DE9F04F8DB0FCF75DFE18B100200DB031
:10B99000BDE8F08F7A4C4FF0000BC4F818B4BFF339
:10B9A0004F8F60680290A568D846284004EB80005D
:10B9B00008E021680298814201D86160E6E72840EA
:10B9C00004EB80000C3002A9FEF740FA0028F0D109
:10B9D00005AA029901EA050304EB8303491CDB680D
:10B9E00042F82030401C02910228F2D3059800F062
:10B9F0000300022802D001284ED0A9E00598502269
:10BA0000810D8946B2EB905F00D850210E4666F357
:10BA10009F50059008315B4800F0E7F9070079D0A6
:10BA200000F02CFA4346082205A9384600F041FAF6
:10BA3000029908F1080A2940681A8000001D864210
:10BA400023D94F4D0C3530B1C2B204EB8101301A0D
:10BA500090460C3104E02946F2B200259046284673
:10BA6000C6B25346384600F024FA0AEB08032DB15B
:10BA7000324629464FEA070000F01BFA029909F105
:10BA8000030001EB900002903BE004EB8101534680
:10BA9000324638460C31EFE70598C0F3831006288C
:10BAA00000D30620059960F38911C1F38310801C2F
:10BAB00005918100334800F098F9070048D000F064
:10BAC000DDF94346082205A9384600F0F2F908F1ED
:10BAD000080800260FE00298434600EA0501401CD2
:10BAE00004EB81010290042238460C3100F0E1F9A8
:10BAF00008F10408761C0598C0F38310B042EAD818
:10BB000047B1D4F81054D4F8180468B1384600F09E
:10BB1000BBF92FE01CE0687A012804D12A68284686
:10BB20003946126890476D68002DF4D1384600F010
:10BB3000ABF98DF800B06846FBF786F9D4F8180425
:10BB400008B9029860609DF80000FBF7A1F911E0C8
:10BB5000D4F8104404E02168204689688847646866
:10BB6000002CF8D108480221008801EB004007A111
:10BB700000F016F8FCF766FD80F0010007E7000012
:10BB8000942D00208C070300242400204261636B65
:10BB9000656E647320666C757368656400000000F0
:10BBA00000231A4603F0D2B808B5012300926A4672
:10BBB00003F0CCF808BD1CB5CDE9002302236A468A
:10BBC00003F0C4F81CBD3EB5069C8DE81C000323A1
:10BBD0006A4603F0BBF83EBD2DE9F0470E468046AD
:10BBE0001C46924608293ED894F80C9000202073F9
:10BBF0001946104602F09AF80025B54206D218F808
:10BC000005201AA12046FFF73DF903E019A12046BF
:10BC1000FFF738F96D1C082DEFD317A12046FFF769
:10BC200031F90025B54210D218F80570FAF71AFC60
:10BC30000068C05D10F03E0F01D03A4600E02E22B1
:10BC40000EA12046FFF71EF903E00DA12046FFF7E5
:10BC500019F96D1C082DE5D301222146504602F04A
:10BC600047F884F80C90BDE8F087000020253032BA
:10BC700078000000202020007C00000025630000E8
:10BC800020000000104810B5FF21816000210160F4
:10BC90004160C0F81814C0F8141480F820140B4840
:10BCA00000F0F0F800280DD109480A490A4B401A63
:10BCB000C108002003E000BF23F82000401C884298
:10BCC000FAD3002010BD0000942D00208C07030043
:10BCD0008C0703000C070300F423002002480349EB
:10BCE000401AC008704700008C0703000C070300CF
:10BCF00013B56846FEF786FC08B100201CBD02485B
:10BD0000009950F831001CBD0C07030070B50848BD
:10BD10000125D0F8104480F8205405E065722168B0
:10BD20002046496888476468002CF7D170BD000040
:10BD3000942D00202DE9FF4781460C9D00200C46E4
:10BD40002F7B2873984616462946184601F0EEFFC9
:10BD5000072E42D2DFE806F004090F161F2A36002C
:10BD600049462846FFF78EF837E0494628462268BC
:10BD7000FFF788F831E0D4E9002349462846FFF769
:10BD800081F82AE0A0680090D4E9002349462846BB
:10BD9000FFF778F821E0D4E90201CDE90001D4E908
:10BDA000002349462846FFF76DF816E004F1080025
:10BDB00007C88DE80700D4E9002349462846FFF765
:10BDC00061F80AE004F108000FC88DE80F00D4E91B
:10BDD000002349462846FFF755F8002229464046E9
:10BDE00001F086FF2F73BDE8FF872DE9F041858ABA
:10BDF00080462D1F4819C01CB0FBF5F0C6B2404666
:10BE0000FEF785FD041E19D000202071012060710D
:10BE1000E58000272546761EC4F800800BE04046EA
:10BE2000FEF775FD60B16179491C617128600546B6
:10BE30007F1CC0F80080B742F1D32046BDE8F081F6
:10BE4000204600F002F80020F8E72DE9F04145799E
:10BE500001466B1E002201E00968521C9A42FBD386
:10BE60000F680146002605E038460C68FEF771FDB4
:10BE70002146761CAE42F7D3BDE8F0810121001DBA
:10BE8000FEF719BDFEF77DBD10B504460121001D6A
:10BE9000FEF737FD10F0FF0F04D12046BDE810403B
:10BEA000FFF7D3BF10BD38B501240094FEF76EFB39
:10BEB00038BD38B500240094FEF768FB38BD00009B
:10BEC0000F4910B500204870091D0860BFF35F8F4F
:10BED0000C490D4800F062FA0A480C4A0121001F83
:10BEE000FAF722FF002809D106480022001F4FF46C
:10BEF00000410068BDE81040FAF752BF10BD0000D5
:10BF00005C230020FCFB0200882C002091BF020073
:10BF100008B500208DF800006846FAF795FFF1EEAD
:10BF2000100A20F09F00E1EE100ABFF35F8F08496E
:10BF30004020C1F880029DF80000FAF7A9FF00F048
:10BF4000FBF908B141DF08BD20BF40BF20BF08BDDD
:10BF500004E000E070B504460C480121FEF7C6FC81
:10BF6000BFF35F8F0025002809D10120074E042C64
:10BF700008D0311F4A781AB1BFF35F8F356070BDAA
:10BF80000C70487002F02EFCF6E7000060230020E1
:10BF900003484078002802D00420FFF7DBBF704739
:10BFA0005C230020FAF76EBE20B1034909680160E6
:10BFB000002070470E207047E8FD0200FEB50246E3
:10BFC0000E460846FFF7F0FF00286ED100250095C9
:10BFD0000195012406208DF80020ADF8040002959B
:10BFE0008DF8024069462020326869DF2F4F48B142
:10BFF00000F018FA3988024604EB01432C49184630
:10C00000FFF7D2FD00958DF801408DF802500195A3
:10C0100002958DF8035069464020326869DF40B1CF
:10C0200000F000FA02463888224904EB0040FFF78E
:10C03000BBFD0095019502958DF8004069460120F1
:10C04000326869DF48B100F0EDF93988024604EB47
:10C05000014319491846FFF7A7FD4FF4B06000905F
:10C06000019502956946A120326869DF48B100F068
:10C07000D9F93988024604EB014310491846FFF705
:10C0800093FD0095019502958DF800406946A0202A
:10C09000326869DF40B100F0C5F9024638880849C6
:10C0A00004EB0040FFF780FD0020FEBD2C240020A3
:10C0B000A8050300F005030008050300540503006C
:10C0C000B40403002DE9F0410446D0F8008060DF9D
:10C0D0002168194D074641451CD92888022606EBE0
:10C0E000004016A1FFF75CFD2888424606EB0040A1
:10C0F0001EA12368FFF75FFDF006D0F80C01216850
:10C10000800200F10050421A288825A106EB004069
:10C11000FFF74AFD012467B1384600F083F9024673
:10C1200028882AA104EB0040FFF73EFD3846BDE811
:10C13000F0812E480470F9E72C240020496E7375B5
:10C140006666696369656E742052414D20616C6C4E
:10C150006F636174656420666F7220746865205334
:10C160006F66744465766963652E00004368616E8E
:10C170006765207468652052414D20737461727444
:10C18000206C6F636174696F6E2066726F6D203012
:10C1900078257820746F20307825782E00000000F4
:10C1A0004D6178696D756D2052414D2073697A65D6
:10C1B00020666F72206170706C69636174696F6E64
:10C1C00020697320307825782E00000073645F6248
:10C1D0006C655F656E61626C652829207265747597
:10C1E000726E65642025732E00000000DB230020A2
:10C1F00030B5144891B00078002820D05FF03405A5
:10C20000ADF8405010A903A861DF30B1052816D061
:10C2100011B0BDE83040FAF735BD03AC0A496846B5
:10C2200000F0BCF807E000BFD0E9002120469047AD
:10C23000684600F0CAF802980028E1D0F4E711B08F
:10C2400030BD0000DB230020ECFD0200F8B5134CEC
:10C250002078C0B10120A07002F06AF8112814D033
:10C26000022002F07DF800258DF800506846FAF7AC
:10C27000EBFD11DF064625709DF80000FAF708FE79
:10C280002EB13046F8BD0820F8BD0020F8BDA570DD
:10C2900002F014FD032002F063F8F6E7D823002033
:10C2A0007CB5194C207808B108207CBD0120A07015
:10C2B000002002F03DF8112819D0002002F050F8BB
:10C2C00012480026006801908DF800606846FAF771
:10C2D000BBFD0F4901A810DF05000AD00020207027
:10C2E0009DF80000FAF7D4FD2DB128467CBD002052
:10C2F0007CBD0120F3E7A670667002F0FBFC012014
:10C3000002F02EF8F3E70000D823002080FD0200A1
:10C31000096C02000EB50749684600F03FF805E0D9
:10C32000D0E900108847684600F04FF802980028CE
:10C33000F6D10EBD9CFD0200014800787047000058
:10C34000D82300200548817819B1007818B1FFF78B
:10C350007DBF08207047FFF7A3BF0000D82300204F
:10C360001FB568464BDF30B1052814D004B0BDE8D6
:10C370001040FAF787BC084901A800F00FF806E062
:10C38000D0E900210098904701A800F01EF803981A
:10C390000028E6D0F4E71FBD08FE0200016009682E
:10C3A0004160AFF3008010B5D0E900215368994295
:10C3B00001D1002104E0D1E90034A34202D01946A2
:10C3C000816010BD08314160F0E7816800290BD021
:10C3D000026892680A44826041684B689A4203D1BD
:10C3E00008314160FFF7DFBF704700000C4A10B50D
:10C3F00002F594730EE0991AC91001EBD17149103E
:10C4000002EBC1010C68844201D90B4602E005D25F
:10C4100001F108029A42EED3002010BD486810BD19
:10C420001CFC020000B5FFF7E1FF002800D1014825
:10C4300000BD000008FC02004058002800D0012088
:10C44000704708B5002242504058009008BDD0F80F
:10C450000403084000D0012070474058002800D055
:10C460000120704708B5002242504058009008BD96
:10C4700008480068012110F0010F08D14FF0E020BA
:10C48000E02280F80024C0F88012C0F800110248B1
:10C490000160704700E100E01805004006490246CF
:10C4A00000200B790BB1852070470A6001220A71C8
:10C4B00000224A7170470000B82200200449012080
:10C4C000086004480168C1F300410029FAD17047AF
:10C4D0000C00004018040040002802D001498001EF
:10C4E0000847704721FB02002DE9F0410E468046C7
:10C4F00001F022F9204D0028404616D0FCF7EEF856
:10C50000284490F858008009032802D001280AD056
:10C5100003E04046FFF702F928B103214046BDE899
:10C52000F041FFF7ABB80221F8E701F011F900285C
:10C5300020D04046FCF7D2F80446104F4FF48070EC
:10C5400007EB840100EB8400D1F8102580B242F0A3
:10C550000102C1F81025FFF729F9002E0AD0404644
:10C56000FCF7BCF855F82000002803D00120A040BB
:10C57000C7F80403BDE8F081F42800200060004003
:10C580002DE9FC41DFF8C080044608EB04000027D9
:10C5900090F930001346C0170E46401C01D0082702
:10C5A0004FE0B0781946C0F340022046FCF772F81D
:10C5B0000546401C44D0B07841071CD4C0070DD0BC
:10C5C00068460094FFF780F8009900EB8100D0F8EE
:10C5D000001721F00201C0F8001707E0002173786E
:10C5E000204600910A460191FEF7C5FF16492046F4
:10C5F0006431FEF7E6F9B078800718D51348317832
:10C6000000EB8500D0F81025114B1A40C0F810251A
:10C610004FF47C524FF4403302EA042203EA014112
:10C620000A43D0F810150A43C0F8102509E008EBBA
:10C630000500327810F8581F41EA8211017000E0BD
:10C6400004273846BDE8FC81F42800200060004043
:10C65000FFC0FCFF10B5FFF761F8002800D00120F3
:10C6600010BD000070B5194D95F86A0008B108209A
:10C6700070BD0020411E2A18401CC0B282F8301044
:10C680003028F8D300242046FBF7F6FF641CE4B200
:10C690000C2CF8D30D490024E0204C66A1F868402A
:10C6A0000B4981F8000401264020891FC1F880024F
:10C6B000C1F800014FF4BE70FFF778F80549F007A4
:10C6C000C1F8040385F86A60204670BDF428002094
:10C6D00006E000E000600040034890F86A0000288F
:10C6E00000D0012070470000F42800200121B1EBA8
:10C6F000507F01D1012070470020704738B50D46AA
:10C7000001F060FB040014D000208DF800006846A2
:10C71000FAF79AFB207928B19DF80000FAF7B8FBE8
:10C72000112038BD0120256020719DF80000FAF726
:10C73000AFFB002038BD10B501F044FB002802D04B
:10C7400000210160017110BD0149024802F094BC52
:10C7500060290020002000402DE9F04105460079C5
:10C7600016460F4600EB40012D4A01EBC00102EBDB
:10C77000810494F82A1011B10820BDE8F0812949FC
:10C7800051F820102868FFF7B9FF08B11120F4E72D
:10C7900039462846FAF796FB666038692060300013
:10C7A0004FF001062FD03F7F4FF48E712868FFF7BE
:10C7B00048FE4FF4A2712868FFF743FE28681A4923
:10C7C000C0F8041328684FEA4711000B40B2002854
:10C7D00006DA00F00F0000F1E02080F8141D03E0FD
:10C7E00000F1E02080F800142868000B40B200F04F
:10C7F0001F0206FA02F14009800000F1E020C0F8B3
:10C800008012C0F8001128680421C0F8001500202B
:10C81000A061E06184F8290044F8140FA675ACE724
:10C82000602900200CFB0200800002002DE9F04787
:10C83000054600790B4600EB400101EBC00023499F
:10C8400001EB8004284600F043F810B11120BDE848
:10C85000F0874FF00008C4F82080A360626184F87C
:10C8600028804FF48E76474631462868FFF7E9FD69
:10C8700028684FF00109C0F808902146286802F0A6
:10C8800097FB606800BBD5F800A00EE094F8280084
:10C8900008B10F2716E031465046FFF7CDFD0028BE
:10C8A000F4D02146504602F083FB216A6069814240
:10C8B000F1D331462868FFF7BFFD0028F9D028687A
:10C8C000C0F80C90C4F814803846C0E760290020F6
:10C8D000007900EB400101EBC000044901EB80004E
:10C8E0004069002800D00120704700006029002026
:10C8F0002DE9F047044600794FF0000900EB4001B4
:10C9000001EBC000254901EB80072068C0F80095C5
:10C91000786880B120682249C0F808132068012196
:10C92000000B40B200F01F0291404009800000F16E
:10C93000E020C0F880112068D0F80C25D0F81485CC
:10C94000D0F80865D0F810554FF0FF31C0F8141535
:10C95000C0F80C152068C0F80815C0F81015501C58
:10C9600002D01046FEF752FEB8F1FF3F02D040461B
:10C97000FEF74CFE681C02D02846FEF747FE701CEE
:10C9800002D03046FEF742FE2068FFF7D4FE87F85B
:10C990002A90C7F80490BDE8F087000060290020C5
:10C9A000840202000149024802F012BC8C290020D6
:10C9B000002000402DE9F0410546164600790F465B
:10C9C000154A00EBC00102EB810494F8201011B16C
:10C9D0000820BDE8F081114951F820102868FFF7C0
:10C9E0008DFE08B11120F4E739462846FAF7A5FA7A
:10C9F0006660386920601EB1397F2846FDF7E6F988
:10CA000028680821C0F800150020A061E06101211C
:10CA1000606184F82010DCE78C29002010FB020004
:10CA20002DE9F04704460E460079204900EBC0008E
:10CA300001EB800517463046FFF758FE30B120461F
:10CA400000F036F820B11120BDE8F0871020FBE798
:10CA50006F61AE604FF49076002731462068FFF793
:10CA600001FD4FF4AC7841462068FFF7FBFC2068DD
:10CA7000AA686969C0F84425C0F8481520680121F2
:10CA80008160686878B9B14649462068FFF7E5FCDF
:10CA9000064641462068FFF7E0FC0643F4D000B1AB
:10CAA0000F27002068613846CEE700008C2900205F
:10CAB0000079054900EBC00001EB800040690028C7
:10CAC00000D00120704700008C2900202DE9F0479C
:10CAD00004460079274900EBC00001EB800720687D
:10CAE0004FF00009C0F80095786880B120682249AD
:10CAF000C0F8081320680121000B40B200F01F02AB
:10CB000091404009800000F1E020C0F880112068C9
:10CB1000D0F80C25D0F81485D0F80865D0F8105559
:10CB20004FF0FF31C0F80C15C0F814152068C0F89C
:10CB30000815C0F81015501C02D01046FEF76FFD06
:10CB4000B8F1FF3F02D04046FEF769FD681C02D0F5
:10CB50002846FEF764FD701C02D03046FEF75FFDEC
:10CB60002068FFF7E8FD87F82090C7F80490BDE83B
:10CB7000F08700008C2900201003020010B550B18E
:10CB800003280CD10220FBF7CFFB002807D0BDE81B
:10CB90001040FAF777B8BDE8104001F061BE10BD53
:10CBA0000078002807D104483B21008876DF002860
:10CBB00001D0FAF767B870472022002070B58D8841
:10CBC000027900EBC5042273C97BA41D012902D0A0
:10CBD000022904D101E0008800E0408820802188FB
:10CBE000608881420FD92846A5DF0126A0B111280F
:10CBF00014D0FFF717FC02460A480BA1008806EB89
:10CC00000040FEF7D1FFA179E079814208D928469A
:10CC1000BDE87040FBF7AABE6671F4E72671F2E743
:10CC200070BD0000F423002073645F626C655F6771
:10CC3000617474635F65786368616E67655F6D7466
:10CC4000755F7265717565737428292072657475D6
:10CC5000726E65642025732E000000007CB50646C8
:10CC60008D88C88806EBC504A41D172800D217209C
:10CC70002188814200D808466080002020712188E8
:10CC80002846B5DF50B1FFF7CDFB02460E48012123
:10CC9000008801EB00400DA1FEF786FF60790028B7
:10CCA00010D1306900280DD01449D1E90201CDE935
:10CCB0000001ADF802506088ADF8040032696946A1
:10CCC000304690477CBD0000F423002073645F620F
:10CCD0006C655F67617474735F65786368616E67C4
:10CCE000655F6D74755F7265706C79282920726557
:10CCF0007475726E65642025732E00004CFA020074
:10CD00007FB51A4D8188AA8891422DD110F8061F4F
:10CD1000022929D14188EA88914225D1017A042942
:10CD200022D0062920D005291ED0841C0020009086
:10CD300002210190029003908DF80010297E19B114
:10CD400001218DF8061001E040F2FD10ADF804005D
:10CD5000A8886946B0DF1128FAD0BDF80400002881
:10CD600002D12046FAF79AFE7FBD00009C280020E1
:10CD700048B1064A0168914205D14068044940180B
:10CD800002D0012800D0032070470000DEC0ADDED5
:10CD900002FEE10E8A7D022A04D90289CB881A4458
:10CDA000D21C02814289C988511AC91E418170472B
:10CDB0002DE9F0410D460221904600F5805629806C
:10CDC00000F10804144F1BE031462046FCF776FDC5
:10CDD00040B1B8F1000F02D0012288F800200228EB
:10CDE00016D004E0A0687969884200D97861288863
:10CDF00061880844C01C2880608804EB80040C34DF
:10CE000031462046FCF76DFD0028DDD1BDE8F081FC
:10CE10004FF480602880F9E71023002008B5002136
:10CE2000009101460823024A0248FEF7A1FA08BD14
:10CE300038FB0200E023002008B5002000900448E1
:10CE40000823044A01680448FEF792FA08BD00006E
:10CE50003823002030FB0200E02300202DE9F05FA2
:10CE60000025DFF80891DFF808B12C464FF00308E1
:10CE7000AA462F46D9F80C0000EB07363046FFF7DC
:10CE800077FF78B3012847D0032862D100204FF400
:10CE9000806200BF56F82010491C0ED004EB8401BC
:10CEA0000BEB8102A8F10100566003221FFA80F803
:10CEB0000BF82120641CA4B24BE0401C9042E9D343
:10CEC0002C48016879B104EB840102200BF82100A1
:10CED0000BEB81014E600881254828304480641C9A
:10CEE000A4B205E007E00221066081804FF0010A4C
:10CEF00045F001052DE004EB840100220BF8212010
:10CF00000BEB810101F110024E6030460831FFF752
:10CF10004FFF45F00205CDE7BAF1000F0CD002201B
:10CF200004EB8401134A0BF821000BEB810112681A
:10CF30004A60641C0881A4B20E480022011D0660EC
:10CF40003046FFF735FF0B48808802280CD00820B8
:10CF500005437F1CBFB2032F8CD3B8F1020F00D260
:10CF60000025E8B2BDE8F09F0420F1E7E0230020AF
:10CF7000902B00203823002001494978FAF7E4BBC0
:10CF800080220020002101F06DBE30B585B00C4636
:10CF900005218DF800101546ADF80200FCF70CFED7
:10CFA000ADF804006846CDE90245FBF73FFF05B048
:10CFB00030BD000070B5054D06460024304655F8DA
:10CFC00024108847641C042CF8D370BD7CFA02003E
:10CFD0003EB5104D002400BF05EB041002F096FB97
:10CFE000641C022CF8D30124502002210094CDE9C6
:10CFF00001100849084BB039A02201F1A00000F04F
:10D00000E1FB08B103203EBD0348401E84700020B0
:10D010003EBD0000F02700206D22002000F06CB91A
:10D0200000F06CB970B504460025C168184A28465E
:10D0300002EB00139B688B4202D102EB001003E06D
:10D04000401C0228F4DB00202178082904D009299B
:10D0500008D0132914D112E0617A89B980B102F0A5
:10D0600065FB0DE0617A59B950B100218160817B87
:10D0700041F00201817307490120087003E0012596
:10D080002046FFF797FF2846BDE8704000F0A2BF9A
:10D09000F02700206C22002000F0E5B908B51388C5
:10D0A0009B0000936B4600F05FF908BD002300F081
:10D0B0005BB938B505460024204609E0817828464A
:10D0C00000F080F810B1052800D003240098401C1F
:10D0D00000906946284602F005FB0028EED134B9DD
:10D0E000284600F0C4F910B1072802D003242046D6
:10D0F00038BD0724FBE71346002200F069B90000A1
:10D100002DE9F0471F0015460E46814604D0072E34
:10D1100005D0082E16D102E00E20BDE8F0878DB1B3
:10D12000022D0FD800F0AEF960B14FF00008314683
:10D13000484602F0BDFA041E06D0207BA8420DD05E
:10D140000F20EAE70720E8E7FF214FF6FF7002F023
:10D15000AFFA041E06D0A0F80090A670607BFF28EE
:10D1600002D00CE01120D8E72946154800F0FCFA5F
:10D17000014620466173FF2913D04FF00108257343
:10D18000617B0F4800F03EFB02000DD0ABB2314690
:10D19000384600F007FAB8F1000F0ED0082E05D07F
:10D1A0000BE002F0B3FADDE70320B6E738886FF052
:10D1B000050101EB8000796888800020ADE7000060
:10D1C000E027002070B5002402F072FA05000BD0B1
:10D1D000686820B100F06FF9040000D003242846ED
:10D1E00002F0A4FA204670BD052070BD70B515464A
:10D1F0000C46072903D0082C01D0072070BD02F08F
:10D2000057FA28B105808470BDE8704002F00EBA6C
:10D21000052070BD7CB50D46072903D0082D01D02F
:10D2200007207CBD002602F043FA040002D06068AB
:10D2300010B11CE005207CBD617B0F4800F0E2FAD4
:10D2400002004FF00000009001908DF8025010D0C5
:10D25000237B2946684600F03DF9684602F0D4F980
:10D26000211D684600F010F90646092801D0304615
:10D270007CBD03207CBD0000E02700204FF6FF713D
:10D28000418001490968084764FA020030B587B057
:10D290001748FBF755FF10B1032007B030BDFBF76F
:10D2A00071FE08B18620F8E700F0CEF90020029068
:10D2B0004CF2070403900EE0694604A8FBF70AFF4E
:10D2C00000988088A0F5404085B204A8FBF7C2FE14
:10D2D000284600F075F902AA04A92046FBF7E1FEF2
:10D2E0000028E9D00349012008700020D5E700009C
:10D2F000398E02006022002000F088B900F08CB95D
:10D3000070B586B014460E46054600F03BF940B1B4
:10D3100005F5404080B20F4A6946FBF7C2FE40B9AE
:10D3200002E0012006B070BD03A96846FBF7D2FEFB
:10D3300008B10020F6E7A570039840882080049883
:10D34000606003988088A0F5404030806846FBF715
:10D3500081FEE6E7642200200248002141608160EE
:10D360007047000060220020F0B587B01D461446CB
:10D3700007460E46FF280AD8084600F003F930B1E8
:10D3800003AA3146384600F0E5F840B902E007202C
:10D3900007B0F0BD01A903A8FBF79CFE08B105206A
:10D3A000F6E7A67001984088208045B18200286881
:10D3B00090420BD302996068F9F758F801E002989F
:10D3C000606003A8FBF746FE0020E1E70420DFE7EA
:10D3D0007FB586B01E460D460446FF282AD8A87899
:10D3E00000F0D0F830B304F54040ADF80000A87864
:10D3F00003AA00F54040ADF8020068680190288853
:10D400000290A978204600F0A5F80528089813D0C6
:10D4100010B108A8FBF7C2FE694603A8FBF77EFE21
:10D42000B0B107281DD0082819D00E2817D0032026
:10D430000AB070BD0720FBE728B108AA694603A817
:10D44000FBF777FEECE7694603A8FBF76EFEE7E71C
:10D450001EB1314603A8FBF734FE0020E8E7112097
:10D46000E6E78620E4E74FF6FF7000F0A9B810B5B4
:10D47000FF2801D9072010BD00F0A8F800F02EF811
:10D48000002010BD00F0F4B870B504460D46807859
:10D4900000F078F858B121882846FBF767FE00288D
:10D4A00004D0072805D0092800D0032070BD07202C
:10D4B00070BD862070BD01B56846FBF76FFE002881
:10D4C00000D0032008BD00000149C978FAF73CB933
:10D4D000802200209BB200F065B8000070B51B4DA3
:10D4E0008AB00020687000904FF6FF7601903046B9
:10D4F00003E0204600F07CF8204600F087F8044660
:10D50000B0421DD004F5404080B26A4602A9FBF744
:10D51000D0FD0A28EDD004F5404080B2FBF7F2FCC4
:10D5200008280FD000280BD005461422084905A86A
:10D53000F8F79CFFADF8184005A80795FFF79EFE89
:10D540000AB070BD01206870FAE700006022002078
:10D5500068FA02007CB5054616460C46084600F0FF
:10D5600011F80020009005F54045019004F5404475
:10D57000A8B2A1B26B463246FBF78CFD002800D062
:10D5800005207CBD07280BD0012809D0082807D02A
:10D59000052805D0062803D0042801D000207047B4
:10D5A0000120704710B503EB83034FF6FF7404EAC4
:10D5B00003138170DB1C99084260018010BD0000DC
:10D5C0000149FBF793B800001028002010B504466D
:10D5D000A0F57F40FF3807D004492046FBF786F8C6
:10D5E000A04201D1012010BD002010BD3028002034
:10D5F00010B50446044900F009FE03492046BDE881
:10D600001040203100F002BE102800200149FDF733
:10D6100095B800003028002070B50A49FDF78EF853
:10D6200004464FF6FF7507E000F02CF838B10549C5
:10D630002046FDF783F80446AC42F5D170BD204684
:10D6400070BD00001028002010B508484021F8F7F0
:10D6500026FF4FF480742146044800F0A5F92146C6
:10D660000248BDE81040203000F09EB9102800208C
:10D67000FF2803D80146024800F0C5B900207047D2
:10D6800010280020FF2803D80146024800F0BBB94B
:10D69000002070473028002010B50C46FBF7D2FF61
:10D6A000FF2804D0024900EB400021F8204010BDC3
:10D6B000402600201CB500F051F908B1F9F7E2FA54
:10D6C0000020009001909DF8000020F07E0040F0C6
:10D6D0000100303020F080008DF8000007208DF828
:10D6E000010010208DF802009DF8030040F00300B7
:10D6F0008DF803009DF8040040F003008DF804004D
:10D70000684600F0E5FA08B1F9F7BCFA034800F002
:10D71000C9FA002801D0F9F7B5FA1CBD65D8020096
:10D720000068012805D0022803D0042801D0002079
:10D7300070470120704700000449084490F9300008
:10D74000082801DB0120704700207047F4280020E2
:10D750000449084490F93000082801D2012070479C
:10D7600000207047F42800202DE9F0410F46060004
:10D7700026D0306820B3706810B3FF2400251CE069
:10D780002946706800F017F948B1FF2C00D12C46EB
:10D79000281B401CB8420ED12046BDE8F081FF2C6A
:10D7A00006D108E02146304600F040F8641CE4B29F
:10D7B000AC42F7D3FF246D1CEDB2B068A842DFD8AD
:10D7C000FF20EAE72DE9F0410400DDE90705069EA8
:10D7D00016D0A9B1A3B100FB05F7974210D8C21D1E
:10D7E000B6EBD20F0CD358B155B1E5602160C4E956
:10D7F000013081B2184600F0D7F80020BDE8F08172
:10D800000720FBE770B504000D460DD0206858B125
:10D81000606848B1FF2D07D000F0F5F820B1E1684D
:10D82000206805FB010070BD002070BD70B50400CC
:10D830000D4611D0206800280ED0606800280BD05B
:10D84000FF2D09D000F0DFF8002805D029466068D8
:10D85000BDE8704000F0E3B870BD002901D001F0D0
:10D8600025B87047F8B5044600781E4D03260E28EB
:10D870001DD2DFE800F0071C0F1C1D1C24351C33D3
:10D880001C352E35288818A106EB0040BDE8F8406D
:10D89000FEF786B96088F9F739FF0246207A0090D2
:10D8A0002888638806EB00401AA1FEF78CF9F8BDC2
:10D8B0000020009060886946FFF7CFFFF8BDFBF7B6
:10D8C00043FB0828FAD00028F8D0BDE8F840F9F763
:10D8D000D9B9BDE8F8400020F9F7F2B82069F2E7BD
:10D8E000A068F0E724240020436F6E6E65637465C2
:10D8F0006420746F20612070726576696F75736C37
:10D900007920626F6E646564206465766963652E54
:10D9100000000000436F6E6E656374696F6E207364
:10D920006563757265643A20726F6C653A20256490
:10D930002C20636F6E6E5F68616E646C653A203098
:10D940007825782C2070726F6365647572653A2053
:10D9500025642E00FBF746BAFBF744BA10B5FFF773
:10D9600095FC88B9FFF734FB70B900F0A1FF58B9F6
:10D9700001F0BCF840B9FBF701FE28B9FBF7E6FE61
:10D9800010B9FCF789F808B1032010BD05484FF61F
:10D99000FF718180002181604170012101700020B0
:10D9A00010BD000070220020002803D0C91DC90846
:10D9B000F8F775BD7047002809D001F00703012270
:10D9C0009A40D2B200EBD1001146FCF73BBC704745
:10D9D0002DE9F0410D46060013D0002401270EE08A
:10D9E00004F0070007FA00F0C1B206EBD400FCF720
:10D9F00029FC10B12046BDE8F081641CA4B2AC4201
:10DA0000EED32846F7E740B100EBD10001F0070262
:10DA1000007801219140084000D001207047F8B5FE
:10DA20000400C1F3C70501F007014FF0010000FA3F
:10DA300001F0C6B20FD0605D30420CD000208DF8EE
:10DA400000006846F9F700FA605DB04360559DF844
:10DA50000000F9F71DFAF8BD2DE9F041044686B043
:10DA600001278088FBF7E6FF6080207800263F4D85
:10DA7000082808D0092820D04FF6FF780A2829D096
:10DA80000B2853D158E0607A10B1012809D04DE03D
:10DA9000A86830B1E168814203D1AE60A088A88057
:10DAA00016E06878E8B3A088A98888423ED1207A39
:10DAB00006283BD100F072FA38E0607A88BBA8688B
:10DAC00078B3E168814231D1AE60E868401EE86019
:10DAD000E6602BE0A878E8B14046FFF7A1FA41469E
:10DAE000404517D10846FFF799FA404512D1AE706C
:10DAF00014216846F8F7D3FC0C208DF80000ADF82F
:10DB00000480ADF8028000272046FBF76BF96846D9
:10DB1000FBF768F9687838B1A088A988884203D1F2
:10DB200000E003E000F03AFA002F1CD006B02046D7
:10DB3000BDE8F041FBF756B9A8780028F6D0AE70E2
:10DB400014216846F8F7ABFC0D208DF80000ADF805
:10DB50000480ADF80280A06802902046FBF742F9ED
:10DB60006846FBF73FF906B0BDE8F081702200205F
:10DB70000349097809B1FCF70BB808207047000089
:10DB8000702200202DE9FF4F2A4883B09946007883
:10DB900092468B46B8B14FF6FF763046FFF740FA13
:10DBA000804600200090244801AA062100680190C8
:10DBB000CDF808D04046FFF771FA00256C1E3746B5
:10DBC000072804D017E0082007B0BDE8F08F052033
:10DBD000FAE700200090A84201D305464746A0423C
:10DBE00001D2044646464046FFF71AFA804601AA8B
:10DBF0000621FFF753FAD8B10528EAD0A8F57F41EE
:10DC0000FF3901D00320DFE70399002001B10F8025
:10DC1000BBF1000F01D0CBF80050BAF1000F01D0DA
:10DC2000AAF80060B9F1000FCED0C9F80040CBE7E8
:10DC30000098D0E7702200208CFA020070B5184ED0
:10DC400086B03078D0B10120B0704FF6FF74204616
:10DC5000FFF7E6F90546A0421DD10020B07014215F
:10DC60006846F8F71CFC0C208DF80000ADF8044065
:10DC7000ADF802406846FBF7B5F80EE0082006B0A4
:10DC800070BD00BFFFF774FF08B10320F7E7284617
:10DC9000FFF7C6F90546A542F4D10020EFE70000E2
:10DCA00070220020084A117821B1D178032903D3CA
:10DCB0000420704708207047044B43F82100491C9A
:10DCC000D1700020704700007022002050280020F2
:10DCD0000349097809B100F03DBE082070470000F3
:10DCE00070220020002801D0FBF77CB870470000AC
:10DCF00010B50C46017A052908D0407A38B1084899
:10DD000008A102682046FDF7BDF800E01AB106A19F
:10DD10002046FDF7B7F82046BDE81040FDF7BFB834
:10DD2000B4230020257300000D0A000038B5C38815
:10DD30000D46044633B114A0009015A216A1284642
:10DD4000FDF7A0F8217A05291CD0607A48B1A08897
:10DD5000FDF7F0FD164951F8202016A12846FDF7E1
:10DD600091F8A0880021FDF7C3FF03461049207AEF
:10DD7000143951F8202001B02846BDE830400EA1EA
:10DD8000FDF780B838BD00001B5B306D000000005F
:10DD90001B5B313B33316D0025734C6F677320641F
:10DDA000726F70706564202825642925730D0A0040
:10DDB000B4230020257300003C25733E2025733AD0
:10DDC000200000000349884201D103487047002029
:10DDD0007047000000200040C02200200146054896
:10DDE00010B50068FCF7DDFC04461C21F8F757FB72
:10DDF000204610BD28FB0200014602480068FCF7DF
:10DE0000F1BC000028FB0200034802490068FCF74F
:10DE1000D3BC000058230020B0FB0200F0B5254D14
:10DE2000254E85B004460027686828B92149306826
:10DE30000831FCF7CCFC686001460078072817D24F
:10DE4000DFE800F0160408080E0E12002046FBF76B
:10DE5000FBFE02E0204601F0F3FC040028D008E0BD
:10DE60002046FAF721FEF8E72046FBF731FAF4E7FF
:10DE70000F2414216846F8F712FBA4F5E8501D386A
:10DE800000D10024019469466868FAF7EFFE6846FD
:10DE9000FAF726FF07496F60002408313068FCF765
:10DEA0008BFC044801210C30FCF72BFD0028BBD172
:10DEB00005B0F0BD1023002028FB02002DE9F04141
:10DEC000234C0025234E207A012730B92248311DEA
:10DED0000068FCF77CFC306038B1022020723168A9
:10DEE000087928B101281ED116E06560BDE8F081EF
:10DEF000D1E90503C01A4FF48052904200D3104676
:10DF0000B7EB900F01D2820800E001220869C968CE
:10DF10001844194429DF03E0D1E90301084428DF4C
:10DF200058B1112812D003213068FAF7E9FE2572A2
:10DF30006560BDE8F041FFF767BF207C0028D5D1C0
:10DF4000BDE8F04100210220FDF7C0B92772CDE7FE
:10DF5000542C002054230020B0FB020010B50121F6
:10DF60000448FCF7B4FC002803D1BDE81040FFF7DB
:10DF700055BF10BD1C23002010B5074C201DFCF719
:10DF800097FC002806D1607C002803D1BDE8104032
:10DF9000FFF794BF10BD0000542C0020084910B5B5
:10DFA00000231A46A1F10800FFF7ECFD30B1052867
:10DFB00004D0002002490C39487010BD0120F9E757
:10DFC0007C22002010B510461A46F8F74FFA0020C0
:10DFD00010BD00002DE9F0471B4F8246002638781F
:10DFE00086B0002821D00024DFF86080A14600BF61
:10DFF00008EB0415A87B810702D410EA0A0F1BD096
:10E000000126284601F012FBB0B14FF6FF71ADF8C2
:10E0100002102988ADF80410862809D007218DF850
:10E02000001002906846FEF7C5FF06B0BDE8F08715
:10E0300006208DF80000F5E7641C022CD8D3002ED2
:10E04000F3D187F80090F0E76C220020F027002041
:10E050002DE9F04707461E481C46154600780E4637
:10E0600070B185B17CB1DFF86C804FF00009A088F9
:10E0700002282BD200EB800118F8210010BB19E018
:10E080000220BDE8F0870520FBE720681FB18188EA
:10E090003A8891420ED11EB101883288914209D14D
:10E0A00080682860206868600A48283000892881D4
:10E0B0000020E6E7A088214600F05EF80028E4D1C1
:10E0C000C4F80090A088401CA080D0E70A20D8E7C0
:10E0D00030230020902B0020F8B505464068244FDF
:10E0E0000C46002648B32349CA68824225D80969EC
:10E0F000814222D3FBF704FFF8B12889398988428D
:10E100001BD1D5E900018A68904216D10020A7F101
:10E11000280200BF00EB800302EB83035B688B42A5
:10E1200005D203F580538B4201D9208011E0401CB9
:10E1300080B20228EED30020F8BD268000960AE0C7
:10E14000009829688068884205D1009868603889FD
:10E1500028810120F8BD2088694600F00DF80028CC
:10E16000EED12088401C80B220800228E6D3E2E76E
:10E17000B82B0020E023002070B50E4600EB800194
:10E18000134800EB81004468306804F5805518B1ED
:10E19000418800EB810411E0083410E02946204654
:10E1A000FBF78CFB20B1012805D0022807D10DE038
:10E1B0000120346070BD608804EB80040C34294673
:10E1C0002046FBF78EFB0028E8D170BD002070BD13
:10E1D000902B002038B50C46002100910146042305
:10E1E000074A0848FDF7C4F808B10E2038BD064AB2
:10E1F00004EB840102EB810101200874002038BD8A
:10E200002CFB0200E0230020902B00200A46FF2870
:10E2100003D801461046FFF702BC70470846704716
:10E2200070B5012670044FF0E0210025C1F880018F
:10E23000084C4010C4F84803C4F8080366602F2057
:10E24000FEF74AF9A660044C2F20A560FEF744F9BA
:10E25000A57070BD00100140E822002070B5054691
:10E2600088690C4600284FF4847128460AD0FEF7CE
:10E27000E8F8D5F81805626AE1688854606A401CBD
:10E28000606270BDFEF7DDF8D5F8180570BD1FB5EA
:10E2900001238DF80030CDE90121D0E90012684654
:10E2A00090471FBD1FB501238DF800308DF8081071
:10E2B0000192D0E90012684690471FBD10B5044690
:10E2C000064841792046F9F73FFA002804D1204654
:10E2D000BDE8104000F0FCB910BD0000482200204D
:10E2E00038B50021012548B101280CD0032809D1F7
:10E2F000FEF7BEF8BDE83840FCF778BD4FF0E020EF
:10E30000C0F8805138BD8DF800106846F8F79CFDC4
:10E31000064C207808B9FCF74DFDE068401CE06031
:10E32000A5709DF80000F8F7B3FD38BDE028002087
:10E330003EB5044609496846FEF730F808E000BFDC
:10E34000D0E900212046904730B16846FEF73DF8FD
:10E3500002980028F4D13EBD11203EBD84FD02008C
:10E360003EB5044608496846FEF718F807E000BFC6
:10E37000D0E90021204690476846FEF726F802982B
:10E380000028F5D13EBD000090FD02002DE9FC41C2
:10E3900004460C3000278046FBF71EFC4FF6FF7545
:10E3A0000646A842208803D1FBF706FC064602E099
:10E3B0003146FBF7EBFB20880022012100F0C6F874
:10E3C000AE4212D06A4607213046FEF76FFE60B9B2
:10E3D000019D95F844003435C00705D1414605F14B
:10E3E0001200FBF7BEFB00B12F46002320881A461F
:10E3F000394686DF05000BD0002320881A463146B7
:10E4000000F088F82088294600F002F9BDE8FC8178
:10E41000002FFBD1002320881A46314600F07AF8FD
:10E420002088002241F20601FAF7F4FBEEE7000033
:10E430002DE9FC411D46089C16460F46804644B116
:10E440006B46012207213846FEF75AFE112801D0FB
:10E4500010B10320BDE8FC8150210198F8F71FF8A6
:10E46000019806700198E5603430206001981830FA
:10E4700020610198401C60610748E06101994046B5
:10E480001131FBF75BFA0028E3D107213846FEF78C
:10E49000C1FE0528DDD0DDE75C280020002835D04E
:10E4A0000278910701D411062FD4C2F30211042976
:10E4B0002BD8930703D5032901D1110625D543781D
:10E4C00081788B4221D8072B1FD310291DD8C17802
:10E4D0004B071AD40079430717D40B0715D4030749
:10E4E00013D4D2074FEAC17201D042B10FE062B932
:10E4F00089070AD4C10708D1800706D407E0890735
:10E5000005D4C10703D1800701D400207047012042
:10E510007047000070B50C4605466AB1002B12D05A
:10E5200009480122C1782846F9F726F921462846EC
:10E53000BDE87040FBF72ABB002B04D0BDE870405B
:10E540000846FBF725BB70BD80220020F0B5174DB3
:10E5500014460F460A4685B006462978F9F70CF9A5
:10E56000002F1FD00CB1012200E000226978304654
:10E57000F9F702F9012C17D00022A9783046F9F7F3
:10E58000FBF80022E9783046F9F7F6F8142208493A
:10E590006846F7F76BFFADF802608DF808406846F3
:10E5A000FAF736FC05B0F0BD0122E6E78022002034
:10E5B000A0FA020010B586B0044614216846F7F7A9
:10E5C0006EFF04208DF80000ADF802406846FAF7AF
:10E5D0001FFC06B010BD000002498969002900D067
:10E5E00008477047AC25002030B585B00C4605467D
:10E5F000142206496846F7F739FFADF8025068461D
:10E600000294FAF7E1FB05B030BD0000DCF902002E
:10E6100030B585B00C460546142206496846F7F722
:10E6200025FFADF8025068460294FAF7F1FB05B0F9
:10E6300030BD0000B4FA020070B50D4C0020D2B21B
:10E640002070201D0B4D0378EB5C1BB1001DFEF705
:10E65000E7F902E00C30FEF7E9F808B1F8F712FB31
:10E660006078002802D021780029FAD070BD00001F
:10E6700064230020A42200200348002201490079DD
:10E68000F9F72EB8BDE20200482200207CB50E4901
:10E690000E4C0022D1E90001CDE900016946A088B5
:10E6A000FEF729FD4FF6FF7507E00846FEF7B8FCB8
:10E6B000A08000226946FEF71EFDA188A94201D074
:10E6C0001128F2D17CBD000030FA02005422002053
:10E6D00070B586B0064601250024FBF7D3F8112853
:10E6E00012D005DCF0B1062828D0082808D125E092
:10E6F000A0F54051023907D0A1F54071FF3924D06F
:10E7000001463046FFF770FF2A46124D3046297900
:10E71000F9F732F8697906B022463046BDE8704014
:10E72000F9F72AB814220C496846F7F79FFEADF8AE
:10E73000026001246846FAF747FBE5E7002530460A
:10E74000FBF73AFAFAF7F4FFDEE73046FBF73EFD57
:10E75000DAE700004822002004FA02002DE9F04127
:10E760000746806A14468846C8B3002531E000BFDA
:10E77000B96A05EB450001EB8006B088801CFE28D5
:10E7800002D90C20BDE8F0812288401C08F8020064
:10E7900020881622401C80B2208008F800202088A3
:10E7A000401C80B2208000EB0801308800F08AFD18
:10E7B0002188084480B22080B28842B1B16871B12A
:10E7C0004044F7F753FE2088B188084420806D1C30
:10E7D000EDB297F82C00A842CAD80020D2E7FFE794
:10E7E0000720CFE770B5194D194C07E00168207874
:10E7F0008847002829D01548FDF7E7FDA8680028BC
:10E80000F4D1FDF783FA00BFFDF7BAF80028FBD179
:10E81000207803280CD002280AD0FDF78DFD00B126
:10E8200033DF0C4901200860BFF34F8F20BFFDE7A5
:10E83000BFF34F8F08480168084A01F4E0611143B3
:10E840000160BFF34F8F00BFFDE770BD882C002033
:10E850005C230020000500400CED00E00400FA05F8
:10E8600010B50020F9F760FD08B1F8F70BFAF9F7D9
:10E87000B5FC08B1F8F706FAFDF7E8FC002803D06C
:10E88000BDE81040F8F7FEB910BD000010B500F06B
:10E89000ABF80548002203494078BDE81040F8F77E
:10E8A0001FBF0000A9A002008822002000F016B9B6
:10E8B00010B51148FAF7A9FC0F48401CFAF7A5FC5F
:10E8C0000D48801CFAF7A1FC0B48C01CFAF79DFC10
:10E8D0000948001DFAF799FC0748401DFAF795FC16
:10E8E0000548401E8179182903D00121C1710020FB
:10E8F00010BD032010BD00008922002010B5007853
:10E90000114C0A2813D004DC082810D009281AD189
:10E910000DE00B280BD0132815D100220B49A0794C
:10E92000F8F7DEFE00220A49A078F8F7D9FE0022A7
:10E9300006496079F8F7D4FE6078BDE810400022FF
:10E940000349F8F7CDBE10BD8822002085CF020014
:10E95000A9A0020070B50B4C05004FF001060CD0C9
:10E96000FFF79CFD58B1286820612879207504F1D3
:10E970001000A0602670002070BD0020F9E707207D
:10E9800070BD00008822002010B5044600780528DC
:10E9900002D0122821D105E06088A168BDE81040AE
:10E9A00000F060B90F480021806880B10D48237ADB
:10E9B0001030007800F0010203B101239A4206D31F
:10E9C000627AC0F3400002B10122904200D20121DC
:10E9D000608801230022FBF7C5FA2046BDE81040FD
:10E9E000FAF724BA8822002030B50446008885B0A2
:10E9F00014284FD00ADC11282CD0132828D134F841
:10EA0000040FF8F783FE01282FD038E0192847D0EB
:10EA10001A281DD1A088FEF7AFFA002818D1A088C7
:10EA2000F8F74EFE0028A0884BD02A49002209782A
:10EA3000F8F7A2FE02208DF80000A088ADF80200D1
:10EA400000208DF808008DF809006846FAF7E0F913
:10EA500005B030BD207A3D2804D04FF48851A088FD
:10EA6000002224E041F23D01F9E72079C00701D0FE
:10EA7000012200E0022220880121FFF767FD34F81F
:10EA8000045B142214496846F7F7F0FCADF8025015
:10EA90000294DAE705B0201DBDE83040FFF776BCF0
:10EAA000217A201D41B14279008802F0030205B0AD
:10EAB000BDE83040FBF7B2BA05B0BDE83040F8F72A
:10EAC00079BA05B00122BDE8304041F20601FAF7FB
:10EAD000A1B8000080220020DCFA02000A78024976
:10EAE0000979F8F749BE00008022002010B51448CB
:10EAF000FAF782FB1248401CFAF77EFB1048801C94
:10EB0000FAF77AFB0E48C01CFAF776FB0C48001D9A
:10EB1000FAF772FB0A48017818290FD041781829B2
:10EB20000CD08178182909D0C178182906D001792C
:10EB3000182903D001214171002010BD032010BD10
:10EB40008022002070B50C460546F8F7DFFD01284D
:10EB500002D043F2020070BD21004FF00000FAD055
:10EB600028467EDF70BD00002DE9F74F8AB092463F
:10EB700088460A98F8F7CAFD06464FF6FF79002442
:10EB80004D4627460A98FEF79FFC8346202101A8A0
:10EB9000F7F785FC012E01D0DEB105E02F480022F9
:10EBA00001790A98F8F7E8FDB8F1000F16D098F847
:10EBB0000000C00714D00A98FAF7FEFF0546484542
:10EBC00016D1FEF769FA054648450ED04FF0010B05
:10EBD0000CE043F202000DB0BDE8F08F852721E084
:10EBE0001F48CDF810A008901CE003246CB121E070
:10EBF000012E0AD10A98F7F7B3FF30B90A98FFF748
:10EC0000D9FC0A98F7F7ACFF50B101A80090534621
:10EC1000324629460A98FFF70BFC040002D009E0AF
:10EC2000852712E0012E10D001AB002239460A9848
:10EC30007FDF044654EA07000DD000225B462946D8
:10EC40000A98FFF767FC2046C5E701AB4246394604
:10EC50000A987FDFEDE70122F0E700008022002024
:10EC60005C2800203EB505460C466846FBF75CFD77
:10EC70006A4621462846FEF788F909480099C26885
:10EC80002846FFF771FF0446014601222846FAF79D
:10EC9000D9FA21462846009AFAF75CF83EBD0000F2
:10ECA00088220020002805D1034901204870002057
:10ECB000F9F738BD70470000E028002010B5162095
:10ECC000F7F7ACFE48B10A4882684FF4800152B1B0
:10ECD000016821F48001016010BDBDE8104042F2DE
:10ECE0000100F7F7CFBF4FF0E020C0F8801110BD52
:10ECF000DC2A002010B51620F7F790FEA0B11148CD
:10ED000090F800044009082811D280B101280ED0E3
:10ED100004280CD00C4882684FF480016AB1016865
:10ED200041F48001016010BD42F2010001E042F2B5
:10ED30000200BDE81040F7F7A5BF4FF0E020C0F893
:10ED4000001110BD16E000E0DC2A00202DE9F84F8C
:10ED5000204D924689460646984601226946184645
:10ED6000AF68F9F717FC58B3009800210446801CDF
:10ED700009E000BF00EA07035AF8212005EB8303EE
:10ED8000401C491CDA604145F4D34FEA164AF9F7B2
:10ED900017FF4AEA0041601C384005EB80003C4008
:10EDA00005EB8402C160D06866F3C50068F3891082
:10EDB00069F39F2020F00300401C20F00400D06085
:10EDC00095F8200402E000BFFCF7DAFD0028FBD133
:10EDD000BDE8F88F942D00202DE9F84F1D4C00253B
:10EDE0006846D4E901A6F9F7F5FE002738B30023F9
:10EDF000009A61681CE0D1F800C00846944503D928
:10EE0000ACEB02020A6015E0A2EB0C02634407605F
:10EE1000D0F80CC0C1698146BCF1000F08D006EBE8
:10EE2000030828F07F48C0E9018CC9F81C5005464A
:10EE30000029E0D128466160FBF74CF903E0284641
:10EE4000FBF748F910B15046F9F78EFCE770BDE8C2
:10EE5000F88F0000E82200200D4B10B5596831B141
:10EE600002680C68A24204D8A21A0A60C161586004
:10EE700010BD0B4603E00B46C969121B21B10C689B
:10EE80009442F8D3A41A0C600260C161D86110BD2D
:10EE9000E82200202DE9F041144E77683D462C46CB
:10EEA00003E0844204D02546E469002CF9D11BE03C
:10EEB000D4B1A5420BD1F869706040B90C4901206A
:10EEC00088600021B160F0702F20FDF705FB2168FC
:10EED000E069E86110B1026811440160706887421E
:10EEE00002D00120BDE8F0810020FBE7E8220020ED
:10EEF000001001407CB5064600240D468DF8004008
:10EF00006846F7F7A1FF01A800F0AEFA70B10570EE
:10EF1000094946609DF8040048709DF80000F7F725
:10EF2000B7FF1420F7F718FC20467CBD04249DF899
:10EF30000000F7F7ADFFF7E7D02900202DE9F041F9
:10EF4000194D6C68002C2CD0184800270068A9685F
:10EF5000B846401A20F07F462068B0420CD82146BF
:10EF6000361A0744E469087C20B181F8108088696A
:10EF700049698847002CEFD129786878814206D109
:10EF8000401CC0B26870022801D185F80180064893
:10EF900069780C3040F82170BDE8F0411420F7F793
:10EFA000DBBBBDE8F0810000E82200200415014031
:10EFB00070B50C4605464FF48E71FDF742FA216A92
:10EFC000A068415C206A401C2062C5F81C1570BD19
:10EFD0001FB500228DF800200291816801914261E5
:10EFE000D0E90012684690471FBD00001FB50A46D1
:10EFF00001788DF8001041680191017A8DF80810B0
:10F00000C0680390044850F82210083850F82220B5
:10F01000684690471FBD0000B02200200149012032
:10F02000087070476423002010B588B00446202281
:10F030000E496846F7F71AFA06200090C01F0190A3
:10F04000029003904FF0EB7006900CB1084A00E07C
:10F05000002269460748FBF7E1FE08B1F7F712FE08
:10F060000448001F447008B010BD000050FD0200AD
:10F070001DF00200682300202DE9FF470C460546DD
:10F080004FF40071FDF7E3F901274FF401780026F2
:10F0900018B34FF4927949462846FDF7CDF9E0B10F
:10F0A00049462846FDF7CDF9C5F8088394F82900AC
:10F0B00000B96F6002208DF80000D5F88004C5F813
:10F0C00080040390A0690290E0680190A661E66167
:10F0D000D4E900126846904728E004212846FDF74D
:10F0E000B6F918B34FF484712846FDF7A5F9E8B1D5
:10F0F00021462846FFF7B2F8616AA069884215D117
:10F10000E06938B1E268616AA0612069E66166621F
:10F11000E06008E094F8290000B96F60C5F8088342
:10F12000A661E268616A2046FFF7B1F84FF48E7875
:10F1300041462846FDF780F978B1206A6169884226
:10F1400002D294F8280020B341462846FDF779F909
:10F15000616911B12046FFF73BFF4FF4A2784146A9
:10F160002846FDF769F9002818D041462846FDF7E2
:10F1700068F994F8290000B12F60A06900280DD02B
:10F18000A661E268616A04B02046BDE8F047FFF777
:10F190007EB821462846FFF70BFFDEE7BDE8FF8774
:10F1A0001FB50A4601788DF8001041680191017A77
:10F1B0008DF80810C0680390044850F822100838F1
:10F1C00050F82220684690471FBD0000B022002062
:10F1D0002DE9FF410C464FF4927705463946FDF77D
:10F1E0003CF90026C0B139462846FDF73BF902201C
:10F1F0008DF80000D5F88004C5F880040390D5F898
:10F200003C058DF80800E0680190A661E661D4E94C
:10F2100000126846904723E04FF488773946284625
:10F22000FDF71BF9E0B139462846FDF71BF9D5F883
:10F230003C15A069884213D1E06960B1E268D5F855
:10F24000000220F02000C5F80002E069A0612069FA
:10F25000E661E06001E0A661E2682046FFF722F87F
:10F260004FF4A27739462846FDF7F7F860B13946E2
:10F270002846FDF7F7F8A06930B1A661D5F83C152E
:10F280002046E268FFF70EF84FF49077394628469B
:10F29000FDF7E3F8002813D039462846FDF7E2F8D9
:10F2A000606900280CD0D5F84C058DF800608DF809
:10F2B0000800A06801906661D4E900126846904792
:10F2C000BDE8FF810870000A487002207047000006
:10F2D00010B514210448F7F7E2F804480068FBF77A
:10F2E00045FA002010BD0000542C0020B0FB0200A5
:10F2F0002DE9F05F8346DDE90A4A994690460D46BE
:10F300000846012703E000BFB0FBF8F07F1C404532
:10F31000FAD2B94500D94F465FEACA7012D18CB112
:10F320005FEA8A7002D5B9F1000F01D0202607E00C
:10F33000302605E031465846641EF9F773F90CB1E2
:10F34000A742F7D35FF00106B9F1010F02D9A9F185
:10F35000010903E0B5FBF6F0404502D306FB08F6D1
:10F36000F2E7DFF83C9000BFB5FBF6F000FB165566
:10F3700019F800105846F9F755F9B6FBF8F6002EC3
:10F38000F2D15FEACA7009D0002C07D0A74205D29B
:10F3900020215846641EF9F745F9F5E7BDE8F09FCE
:10F3A00040FB02000348002201498078F8F798B931
:10F3B000298A020048220020F8B5054680B2FAF7F3
:10F3C000A7FC040013D0154E207A0027317B884219
:10F3D0000ED2A8B204F10A0175DF28B1112806D0B7
:10F3E000BDE8F840FFF7F8B8207A401C2072F8BD5D
:10F3F0002772307C38B1A8B23B2176DF18B10828DB
:10F4000001D0FFF7E9F871690029F0D08DF800709C
:10F41000ADF8025068468847F8BD0000AC250020D2
:10F42000417939B190F8B21021B990F8B40008B11F
:10F43000012070470020704701460148FBF71DBAC4
:10F44000C825002030B40446007A00280AD060881D
:10F45000002166DF28B1112802D0616830BC08475E
:10F460000120207230BC70470A494A788B78521CC0
:10F47000D2B2934200D100220B78934201D10020F6
:10F4800070470270487800EB400001EBC000001D9F
:10F4900070470000D02900202DE9FC411646DDE927
:10F4A0000854CDE900541F468046022200F00CF8B3
:10F4B000002807D1CDE900543B4610223146404692
:10F4C00000F002F8BDE8FC812DE9FC5F0026DDE9D3
:10F4D0000C4B994692468E4680462788354630E04A
:10F4E000D8F80400002200EB85006946006801900E
:10F4F00001A864DF002830D19DF8000050451FD1DD
:10F500000EB1002100E0022122880844111859455B
:10F5100022D846B9521C90B2208009F800E0208819
:10F52000401C20800126218801A801EB09026946C0
:10F5300064DF002811D120889DF800100844208045
:10F540006D1CB8F80000A842CADC56B12088C01B68
:10F55000401E80B2FF2802D90C20BDE8FC9F09F8AC
:10F5600007000020F9E7000010B504281DD209B1FA
:10F57000032400E00024F8F773FD202802D24FF0A6
:10F58000A04102E00A4900F01F0001EB8000D0F822
:10F59000001721F44031C0F80017D0F8001741EAF5
:10F5A0000441C0F80017002010BD062010BD000067
:10F5B00000030050002070472DE9F84F114D884698
:10F5C00081461E4617466946DDF828A02868FBF7E5
:10F5D000E8F8040013D01C21F6F761FF0020207129
:10F5E000C4F80090C4E90486C4E902A76946286803
:10F5F000FBF7F8F8FEF7C0FC0020BDE8F88F042008
:10F60000FBE70000B0FB020082780121012A0BD049
:10F61000062A09D0072A06D0082A06D14168898817
:10F620000931890800E01421018070471CB50446A7
:10F63000002000900190A0788DF80200617B1A48AC
:10F64000FEF7E0F8020017D0237BA1786846FDF7AB
:10F6500041FF6846FFF7D8FF208804F10803694698
:10F660006268FDF7B5FE48B1072806D001210F4AB0
:10F67000112808D086280FD003201CBDA17B21F0C3
:10F680000301A1731CBDA07B20F0010040F002002B
:10F69000A073117000201CBDA37B23F0020343F074
:10F6A0000103A37311701CBDE02700206C22002011
:10F6B00038B505460C46002001E00098401C00903B
:10F6C0006946284600F00EF800280AD08178A14249
:10F6D000F3D1817B8A07F0D4C907EED18168002974
:10F6E000EBD138BD10B5084B0A6809E003EB0214F2
:10F6F0002488844203D103EB02100A6010BD521C1F
:10F70000022AF3D3002010BDF02700204FF6FF712E
:10F710000180FF2181704173817B21F0030181739E
:10F7200000210173416081607047000070B505469B
:10F73000002406E0687B2044C1B20648FEF776F854
:10F74000641C287BA042F5D82846BDE87040FFF72E
:10F75000DDBF0000E02700202DE9FC4706463648C3
:10F760009846144600780D464FF0000978B37DB3F3
:10F770002888A0F57F41FF3931D0688848B3686890
:10F78000FAF7BEFB68B374B32088ADF80000678851
:10F7900001A8FEF723FB04002FD084F800804FF06F
:10F7A000000A84F816A0BDF80000A08268682061F5
:10F7B000214801210C38FBF77EF8E0602888208181
:10F7C0006888A080E780B8F1030F1DD020E001E039
:10F7D00003E004E00220BDE8FC870520FBE70420ED
:10F7E000F9E70320F7E7FFE72889694687B238463B
:10F7F00000F0ACF80028EED1CAE7BDF8001038469A
:10F8000000F098F80820E6E70420A0753068A061B1
:10F81000A4F80A9001A8FEF7EFFA46B1C6F804A0D2
:10F82000E1680648316086F80AA000893081FEF759
:10F8300095FB0020CFE7000030230020B82B0020EC
:10F840002DE9F8430D46898A374A01EB810102EB25
:10F85000810630B129463046FDF79CFA0120BDE80B
:10F86000F88331897068002400EB81072E48A97D58
:10F87000A8384FF00E0807294ED2DFE801F00D2D11
:10F88000162404404A004460A969016026482749BB
:10F89000A838FEF721FC30B10220A87504233946B0
:10F8A0002A1D009423E00A20D9E728692A4608B1D6
:10F8B000032000E001209075042305F10C0207F1FC
:10F8C0000801009413E00120A8750094E88807F16E
:10F8D0000C0183002A690AE028782A4603280CD004
:10F8E00006209075042305F10802391D0094104884
:10F8F000FBF73EFDA8B144460FE00520F1E70621E5
:10F90000A9750A4940680988FEF764FC040004D11F
:10F9100007E041F61D5400E00F2429463046FDF76C
:10F9200039FA20469BE70000902B0020102300208E
:10F93000E023002001EB8102034901EB82014A89A7
:10F94000101AC01E48817047902B002070B5C01C53
:10F9500082B240F2FE30824201D3092070BD114BC9
:10F9600000204FF4806500BF00EB800413F8246092
:10F9700096B903EB84063489768914443444A4B2DE
:10F98000AC4209D2088000EB800003EB8000418983
:10F9900011444181002070BD401C80B20228E3D395
:10F9A000072070BD902B00200D0E0F100B0C1819A6
:10F9B0000C2500202C250020582500200B000300DA
:10F9C000FD8102000C000300FD810200180003000D
:10F9D000FD81020019000300FD8102000700000004
:10F9E0000000000000000000000000000000000017
:10F9F0000600000000000000000000000000000001
:10FA000000000000100000000000000000000000E6
:10FA100000000000000000001100000000000000D5
:10FA200000000000000000000000000001000000D5
:10FA3000010001002CFA02000100010040FA02005E
:10FA40000000000059D902004D950200770A00001D
:10FA500000000000770A0000000000007ADA0000D1
:10FA60000000000025D00200070000000000000098
:10FA700000000000000000000000000059DA020051
:10FA8000FDE802004D980200CD9502000100000043
:10FA900000000000010006007C22002089E902002D
:10FAA0000100000000000000000000000000000055
:10FAB000000000000700000000000000000000003F
:10FAC0000000000000000000030000000000000033
:10FAD0000000000000000000000000000500000021
:10FAE0000000000000000000000000000000000016
:10FAF000E5DC020050EADA308883B89F604F15F3E6
:10FB00000000C98E000000500003005049C70200E9
:10FB1000A5C9020003000000B02900200000000079
:10FB20000338FDD870470000FC2200200000FFFFD2
:10FB3000DEC0ADDEFF011EF1DEC0ADDEFE011EF156
:10FB40003031323334353637383941424344454613
:10FB50006E72665F6673746F726167655F696E6906
:10FB600074006E72665F6673746F726167655F754D
:10FB70006E696E6974006E72665F6673746F72612F
:10FB800067655F72656164006E72665F6673746F4D
:10FB9000726167655F7772697465006E72665F6631
:10FBA00073746F726167655F6572617365000000F1
:10FBB00040230020001000000400000001000000AD
:10FBC000159C0200D1F20200C5DF0200B9F5020067
:10FBD000218C02001DE20200B5F50200999E020090
:10FBE000A4070300A80703000000000000000000B5
:10FBF0000000000000000000682C0020E0FB020074
:10FC0000F8FB020004000000556E6B6E6F776E20EB
:10FC10006572726F7220636F6465000000000000FF
:10FC2000D80303000100000084020300020000006A
:10FC30007800030003000000F80203000400000045
:10FC40004C030300050000002C0203000600000026
:10FC5000C80103000700000034030300080000008F
:10FC60004002030009000000A40203000A00000093
:10FC7000C00303000B000000600003000C00000044
:10FC8000580203000D000000280403000E000000CD
:10FC9000240303000F0000006003030010000000B5
:10FCA00094030300110000003C0403001200000054
:10FCB0001004030013000000AC03030080000000E8
:10FCC000E0010300810000001C010300820000002D
:10FCD000DC00030083000000BC000300840000007F
:10FCE000F800030085000000040203008600000005
:10FCF0000C03030090000000A80103009100000025
:10FD00009C000300920000006C02030000820000CF
:10FD10007403030001820000C0020300028200009D
:10FD2000DC020300008400003801030001840000AD
:10FD3000E403030002840000800103000384000048
:10FD40005C0103001DB90200F1B80200E9B802002D
:10FD5000FFFFFFFFFFFFFFFFFFFFFFFFFFFFFFFFB3
:10FD600000000000000000000000D60107010000B4
:10FD7000F0070300F8070300000000000000000087
:10FD80000100000770FD020080FD02000800000075
:10FD9000A8FD0200B8FD020008000000B8FD020046
:10FDA000C8FD020008000000280803004008030006
:10FDB00000000000000000001808030028080300ED
:10FDC0000000000000000000A8070300B0070300C7
:10FDD000B0070300D8070300D8070300E8070300B3
:10FDE000E8070300F007030020220020C8FD0200FE
:10FDF000E8FD020008000000F807030008080300FF
:10FE00000808030018080300F8FD020008FE0200BD
:10FE10000800000000404040404040404040414118
:10FE200041414140404040404040404040404040CF
:10FE30004040404040050202020202020202020269
:10FE40000202020202202020202020202020200266
:10FE500002020202020290909090909010101010F6
:10FE60001010101010101010101010101010101092
:10FE70000202020202028888888888880808080826
:10FE800008080808080808080808080808080808F2
:10FE9000020202024000000015FE020073645F626D
:10FEA0006C655F6761705F646174615F6C656E67EC
:10FEB00074685F75706461746528292028726571A3
:10FEC0007565737429206F6E20636F6E6E65637441
:10FED000696F6E20307825782072657475726E6552
:10FEE000642025732E0000005468652072657175CA
:10FEF000657374656420636F6D62696E6174696FA8
:10FF00006E206F6620545820616E64205258207015
:10FF100061636B6574206C656E67746873206973C8
:10FF200020746F6F206C6F6E6720627920257520BA
:10FF30006D6963726F7365636F6E64732E0000008A
:10FF400054686520626F6F746C6F616465722068BD
:10FF500061732077726974652070726F7465637461
:10FF60006564206974732073657474696E677320A7
:10FF7000706167652E20546869732070726F6869BC
:10FF8000626974732073657474696E672074686540
:10FF9000206164766572746973696E67206E616D45
:10FFA000652E2054686520626F6F746C6F616465A4
:10FFB00072206D75737420626520636F6D70696C5B
:10FFC00065642077697468204E52465F424C5F53E7
:10FFD000455454494E47535F504147455F50524F37
:10FFE000544543543D3020746F20616C6C6F772012
:10FFF00073657474696E67207468652061647665E2
:020000040003F7
:1000000072746973696E67206E616D652E00000001
:10001000616464725F69735F77697468696E5F6257
:100020006F756E647328705F66732C2070616765EE
:100030005F616464722C20286C656E202A20705FDA
:1000400066732D3E705F666C6173685F696E666F84
:100050002D3E65726173655F756E697429290000B4
:100060004E52465F4552524F525F494E56414C499F
:10007000445F4441544100004E52465F4552524F46
:10008000525F534F46544445564943455F4E4F5483
:100090005F454E41424C4544000000004E52465FD1
:1000A0004552524F525F464541545552455F4E4F5F
:1000B000545F454E41424C45440000004E52465F5D
:1000C0004552524F525F4D555445585F554E4C4F17
:1000D000434B5F4641494C45440000004E52465F49
:1000E0004552524F525F4D555445585F4C4F434B0C
:1000F0005F4641494C4544004E52465F4552524F7F
:10010000525F4D555445585F434F4E445F494E49E9
:10011000545F4641494C4544000000004E52465F42
:100120004552524F525F4D555445585F494E4954C0
:100130005F4641494C4544004E52465F4552524F3E
:10014000525F424C455F495053505F52585F504B8D
:10015000545F5452554E4341544544004E52465FFD
:100160004552524F525F424C455F495053505F5089
:100170004545525F52454A454354454400000000FE
:100180004E52465F4552524F525F424C455F495076
:1001900053505F4C494E4B5F444953434F4E4E457D
:1001A00043544544000000004E52465F4552524FB2
:1001B000525F4150495F4E4F545F494D504C454D41
:1001C000454E5445440000004E52465F4552524F42
:1001D000525F4E4F545F535550504F525445440058
:1001E0004E52465F4552524F525F4D4F44554C451B
:1001F0005F4E4F545F494E495449414C495A45441A
:10020000000000004E52465F4552524F525F4D4F24
:1002100044554C455F414C52454144595F494E4914
:100220005449414C495A4544000000004E52465F33
:100230004552524F525F4E4F545F464F554E440009
:100240004E52465F4552524F525F494E56414C49BD
:10025000445F5354415445004E52465F4552524FFD
:10026000525F444154415F53495A45004E52465FE4
:100270004552524F525F494F5F50454E44494E4799
:10028000000000004E52465F4552524F525F535697
:10029000435F48414E444C45525F4D495353494E8C
:1002A000470000004E52465F4552524F525F494E42
:1002B00056414C49445F4C454E47544800000000AD
:1002C0004E52465F4552524F525F4452565F54570A
:1002D000495F4552525F414E41434B004E52465F8B
:1002E0004552524F525F4452565F5457495F4552F0
:1002F000525F444E41434B004E52465F4552524F6F
:10030000525F494E5445524E414C00004E52465F9A
:100310004552524F525F53544F524147455F4655E5
:100320004C4C00004E52465F4552524F525F4E5564
:100330004C4C00004E52465F4552524F525F494E60
:1003400056414C49445F504152414D004E52465F28
:100350004552524F525F4E4F5F4D454D00000000D9
:100360004E52465F4552524F525F464F52424944A9
:1003700044454E004E52465F4552524F525F4452E2
:10038000565F5457495F4552525F4F56455252553A
:100390004E0000004E52465F4552524F525F494E4A
:1003A00056414C49445F4144445200004E52465F1E
:1003B0004552524F525F5245534F55524345530099
:1003C0004E52465F4552524F525F494E56414C493C
:1003D000445F464C414753004E52465F535543439A
:1003E000455353004E52465F4552524F525F424C66
:1003F000455F495053505F4348414E4E454C5F4125
:100400004C52454144595F455849535453000000EC
:100410004E52465F4552524F525F434F4E4E5F43DE
:100420004F554E54000000004E52465F4552524F09
:10043000525F54494D454F55540000004E52465F9F
:100440004552524F525F4255535900007761726EC8
:10045000696E670064656275670000001B5B313B75
:1004600033306D001B5B306D000000001B5B313BC7
:1004700033316D001B5B313B33326D001B5B313B15
:1004800033336D001B5B313B33346D001B5B313B01
:1004900033356D001B5B313B33366D001B5B313BED
:1004A00033376D00696E666F000000006572726F11
:1004B0007200000073645F626C655F6366675F7300
:1004C000657428292072657475726E6564202573C1
:1004D000207768656E20617474656D7074696E67ED
:1004E00020746F2073657420424C455F474154541B
:1004F000535F4346475F534552564943455F434820
:10050000414E4745442E000073645F626C655F6333
:1005100066675F73657428292072657475726E65ED
:1005200064202573207768656E20617474656D7032
:1005300074696E6720746F2073657420424C455F48
:10054000434F4D4D4F4E5F4346475F56535F5555A2
:1005500049442E0073645F626C655F6366675F7316
:10056000657428292072657475726E656420257320
:10057000207768656E20617474656D7074696E674C
:1005800020746F2073657420424C455F474154547A
:10059000535F4346475F415454525F5441425F5357
:1005A000495A452E0000000073645F626C655F630A
:1005B00066675F73657428292072657475726E654D
:1005C00064202573207768656E20617474656D7092
:1005D00074696E6720746F2073657420424C455FA8
:1005E000434F4E4E5F4346475F4741502E00000049
:1005F00073645F626C655F6366675F736574282907
:100600002072657475726E65642025732077686545
:100610006E20617474656D7074696E6720746F20EC
:1006200073657420424C455F4741505F4346475FC6
:10063000524F4C455F434F554E542E006E72665FCD
:10064000626C655F6761747400000000636C6F63C7
:100650006B000000434C4F434B0000004750494F94
:1006600054450000505253005541525400000000C0
:10067000554152544500000061746669666F2E6DE5
:100680005F717565756500006E72665F6673746F85
:10069000726167650000000061746669666F2E6DA7
:1006A0005F6669666F0000007077725F6D676D74DA
:1006B0000000000062616C6C6F632E6C6F675F6D91
:1006C000656D706F6F6C0000617070006E72665FB8
:1006D000736468006E72665F7364685F626C650065
:1006E0006E72665F7364685F736F63004008030037
:1006F000202200201402000020650200A008030050
:1007000034240020842D00000C6A02003C06030003
:10071000000003034C060300000000005406030021
:10072000000000005C0603000000000064060300F7
:1007300000000000680603000000000070060300CF
:100740000000000078060300000000038806030094
:10075000000003039806030000000003A80603003E
:1007600000000000B406030000000003C8060300F8
:1007700000000303CC06030000000303D4060300BB
:1007800000000303E00603000000030390230020A1
:100790008823002090230020D42C00202024002037
:1007A000180000009D6C0200257F02000000000080
:1007B000F9A90200342400204F73020054240020C1
:1007C000B97D020000000000297E02000000000048
:1007D00029800200000000007BAB020048240020BA
:1007E000E97902009C280020517D020000000000F1
:1007F00095B2020000000000A5EC0200000000001D
:10080000CDB2020000000000B973020054240020A1
:10081000717B020000000000F1C102000000000036
:1008200061C30200000000006186020000000000B9
:10083000E1E2020000000000ADB202000000000092
:10084000062BFFFF0A1801042D55D9022A18017939
:1008500009390A01791310240240200A1A18441297
:1008600020AA4008042544FD0214AC04031A4C04D9
:100870001AA4041A54041A64041A5C041A6C041AA4
:1008800074041A7C041A84041A8C041A94041A9CA2
:1008900004515B90D009210B24C9926C0124000003
:02000004000FEB
:10F0000079CAEF4701000000010000000100000084
:10F010000000000000000000A0A800006FD4D1A9EB
:10F0200001000000000000000000000000000000DF
:10F0300000000000000000000000000000000000D0
:10F0400000000000000000000000000000000000C0
:0CF05000000000000000000000000000B4
:00000001FF
